:10000000C7C70000F0C70000EEC70000ECC7000043
:10001000EAC70000E8C70000E6C70000E4C7000028
:10002000E2C70000E0C70000DEC70000DCC7000038
:10003000DAC700000C942C0AD6C70000D4C7000011
:100040000C949D14D0C70000CEC70000CCC70000A0
:10005000CAC70000C8C70000C6C70000C4C7000068
:10006000C2C70000C0C70000BEC70000BCC7000078
:10007000D92DF42D742E842FA32FCB2FD32F6E2F99
:10008000443A206D61633A2025783A25783A2578FC
:100090003A25783A25783A25780A00443A20656E60
:1000A0006332386A3630207265766973696F6E2004
:1000B000307825780A00443A2064697361626C697B
:1000C0006E67207761746368646F670A00443A2042
:1000D000457468657273657820302E322028292097
:1000E000284465627567206D6F6465290A000022E7
:1000F000F901812600443A206E6F7420656E6F7599
:10010000676820737061636520666F722073746F17
:1001100072696E6720272563270A0025730A000A83
:1001200000443A206D616C6C6F6328292066616918
:100130006C6564210A00443A204552524F523A20DD
:100140007370692074696D656F7574207265616381
:10015000686564210D0A00000123296A285C284E85
:1001600028322827282529D62625303278002578D8
:100170000046757365733A206C6F773D25303258B1
:1001800020686967683D253032582065783D253004
:100190003258006E6574696F5F6164646F6E00440D
:1001A0003A206E65743A207061636B657420746FD9
:1001B0006F206C61726765206F7220746F6F20739F
:1001C0006D616C6C20666F7220616E20657468656D
:1001D000726E6574206865616465723A2025640AF0
:1001E00000443A206E65743A207472616E736D69D2
:1001F00074206572726F72210A00443A206E657431
:100200003A2072656365697665206572726F722146
:100210000A00443A206E65743A207061636B65741D
:10022000207472616E736D6974206661696C6564B7
:100230000A00443A206E65743A206E6F206C696E35
:100240006B210A00443A206E65743A20676F74206F
:100250006C696E6B210A00443A206E65743A207412
:10026000696D656F75742077616974696E67206662
:100270006F722054585254532C2061626F7274690B
:100280006E67207472616E736D6974210A000203D7
:10029000080B1703080308001010202001010002BA
:1002A00003080B1703080308000000000001010009
:1002B00007070B070B000000000107070D0D0000EA
:1002C000010F03070307000000000000010B1100ED
:1002D0000103443A206C63642074696D656F757422
:1002E000210A00443A2073645F7265616465723A62
:1002F000206661745F77726974655F6469725F65B7
:100300006E7472793A20696C6C6567616C207061FB
:1003100072616D732066733D25702C206469725F75
:10032000656E7472793D25700A00443A2073645FEB
:100330007265616465723A206661745F63726561BB
:1003400074655F66696C653A2066696C6520257323
:10035000207375636365737366756C6C7920637263
:1003600065617465642E0A00443A2073645F7265A7
:10037000616465723A206661745F63726561746579
:100380005F66696C653A206661745F77726974654F
:100390005F6469725F656E747279206661696C650D
:1003A000642E0A00443A2073645F7265616465726A
:1003B0003A206661745F6372656174655F66696C3B
:1003C000653A206661745F66696E645F6F66667326
:1003D00065745F666F725F6469725F656E7472796F
:1003E000206661696C65642E0A00443A2073645F7C
:1003F0007265616465723A206661745F63726561FB
:1004000074655F66696C653A2066696C652065781D
:10041000697374732E0A00443A2073645F726561D5
:100420006465723A206661745F6372656174655FCA
:1004300066696C653A20696E76616C6964207061EA
:1004400072616D65746572732E0A00443A2073649C
:100450005F7265616465723A206661745F6F706592
:100460006E5F66696C653A20756E61626C652074BA
:100470006F20616C6C6F63617465206661745F6688
:10048000696C655F7374727563742E0A00443A2058
:1004900073645F7265616465723A20496E6974695C
:1004A000616C697A65642053442D436172642C2029
:1004B0006275742063616E6E6F74206F70656E205C
:1004C000706172746974696F6E2E0A00443A207309
:1004D000645F7265616465723A207265616420745C
:1004E000696D656F75742072656163686564210A62
:1004F00000443A2073645F7265616465723A2066F5
:1005000061696C656420746F2073657420626C6F20
:10051000636B2073697A6520746F203531322062F5
:10052000797465732E0A00443A2073645F726561C2
:100530006465723A2074696D656F757420776169BE
:1005400074696E6720666F72206361726420746FD5
:10055000206265636F6D652072656164792E0A00A3
:10056000443A2073645F7265616465723A20666F15
:10057000756E64204D4D4320636172640A00443AF5
:100580002073645F7265616465723A20666F756E90
:1005900064205344203120636172640A00443A208D
:1005A00073645F7265616465723A2070696E67207A
:1005B000726573756C743A2025640A00443A20739E
:1005C000645F7265616465723A20706572666F720D
:1005D0006D696E672073645F70696E67202E2E2EC2
:1005E0000A00443A205646532D53443A2046616946
:1005F0006C656420746F2063726561746520646942
:100600007220272573270A00443A205646532D535B
:10061000443A20272573272069736E2774206120B0
:100620006469726563746F72792E0A00443A2056C9
:1006300046532D53443A206661745F6F70656E5F58
:10064000646972206661696C65642E202065656B43
:100650002E0A00443A2073645F7265616465723AE1
:100660002053442D4361726420696E697469616C22
:10067000697A656420616E6420726F6F74206E6F9A
:100680006465206F70656E65642E0A00443A2073BD
:10069000645F7265616465723A2053442D436172F0
:1006A0006420696E697469616C697A65642C206282
:1006B0007574206661696C656420746F206F706565
:1006C0006E20726F6F74206E6F64652E0A0025684D
:1006D00068752E256868752E256868752E256868EA
:1006E000750025752E25752E25752E25750025730B
:1006F000007061727365206572726F72003C2144F4
:100700004F43545950452073766700696D616765A2
:100710002F7376672B786D6C003C21444F435459FE
:1007200050452068746D6C006170706C6963617411
:10073000696F6E2F7868746D6C2B786D6C003C3F20
:10074000786D6C00746578742F786D6C002F2A209A
:1007500058504D00696D6167652F782D78706D690F
:10076000003C21444F43545950452068746D6C003F
:10077000746578742F68746D6C003C686561640002
:100780003C7469746C65003C68746D6C003C212D90
:100790002D003C683100503100696D6167652F782C
:1007A0002D706F727461626C652D6269746D617019
:1007B00000503200696D6167652F782D706F72741B
:1007C00061626C652D677265796D617000503300F0
:1007D000696D6167652F782D706F727461626C65E9
:1007E0002D7069786D6170005034005035005036BE
:1007F0000049494E3100696D6167652F782D6E693A
:100800006666004D4D00696D6167652F74696666A7
:100810000049490047494639347A00696D61676586
:100820002F782D756E6B6E6F776E004647463935A3
:1008300061005042460047494600696D6167652F77
:1008400067696600696D6167652F6A706567004258
:100850004D00696D6167652F782D6D732D626D7028
:100860000089504E4700696D6167652F706E6700A3
:10087000464C5600766964656F2F782D666C76005D
:10088000746578742F706C61696E0025750A002597
:10089000750A00485454502F312E31203230302008
:1008A0004F4B0A436F6E6E656374696F6E3A2063D7
:1008B0006C6F73650A00436F6E74656E742D5479A6
:1008C00070653A20746578742F6373733B20636896
:1008D00061727365743D7574662D380A0A00436F42
:1008E0006E74656E742D547970653A2074657874F1
:1008F0002F68746D6C3B20636861727365743D751D
:1009000074662D380A0A00436F6E74656E742D5438
:100910007970653A206170706C69636174696F6E9B
:100920002F7868746D6C2B786D6C3B2063686172F6
:100930007365743D7574662D380A0A0043616368F7
:10094000652D436F6E74726F6C3A206E6F2D63610C
:100950006368650A43616368652D436F6E74726FE7
:100960006C3A206D7573742D726576616C69646183
:1009700074650A436F6E74656E742D547970653AB0
:1009800020746578742F706C61696E3B20636861B8
:10099000727365743D7574662D380A0A00485454A4
:1009A000502F312E31203430302042616420526586
:1009B00071756573740A436F6E6E656374696F6EEB
:1009C0003A20636C6F73650A436F6E74656E742DA5
:1009D000547970653A20746578742F706C61696E13
:1009E0003B20636861727365743D7574662D380AC7
:1009F00000436F6E74656E742D456E636F64696E2F
:100A0000673A20677A69700A004261642052657112
:100A1000756573740A00485454502F312E312034B8
:100A200030342046696C65204E6F7420466F756EB9
:100A3000640A436F6E6E656374696F6E3A20636C0F
:100A40006F73650A436F6E74656E742D54797065AB
:100A50003A20746578742F706C61696E3B2063680E
:100A600061727365743D7574662D380A0046696C51
:100A700065204E6F7420466F756E640A00436F6E7A
:100A800074656E742D4C656E6774683A20000A00B8
:100A90006964782E68740065636D643F0065636DFA
:100AA000643F00474554202F00436F6E74656E7499
:100AB0002D547970653A2025530A0A00256C750A71
:100AC000003C21444F43545950452048544D4C203C
:100AD0005055424C494320222D2F2F5733432F2F5F
:100AE0004454442048544D4C20332E322046696EE5
:100AF000616C2F2F454E223E3C68746D6C3E3C620B
:100B00006F64793E3C68313E496E646578206F665B
:100B10002025733C2F68313E3C7461626C653E3C1D
:100B200074723E3C74683E4E616D653C2F74683E45
:100B30003C74683E53697A653C2F74683E3C2F7460
:100B4000723E0A003C74723E3C74643E3C61206814
:100B50007265663D272573273E506172656E74206D
:100B60004469726563746F72793C2F613E3C2F74E7
:100B7000643E3C74643E2D3C2F74643E3C2F747282
:100B80003E003C2F7461626C653E3C68723E3C6185
:100B90006464726573733E596F757220667269651D
:100BA0006E646C792045746865727365782048546A
:100BB0005450207365727669636520776974682084
:100BC00056465320616E64206D6F645F6D34203A29
:100BD0002D293C2F616464726573733E3C2F626FF4
:100BE00064793E3C2F68746D6C3E003C74723E3CF0
:100BF00074643E3C6120687265663D272573273E1C
:100C000025733C2F613E3C2F74643E3C74643E254A
:100C10006C643C2F74643E3C2F74723E0A003C743A
:100C2000723E3C74643E3C6120687265663D2725D7
:100C3000732F273E25733C2F613E3C2F74643E3C4E
:100C400074643E2D3C2F74643E3C2F74723E004809
:100C50005454502F312E31203330312052454449E5
:100C6000524543540A4C6F636174696F6E3A202594
:100C7000732F0A0A00706F72742025643A2030784E
:100C8000253032780025326868783A2532686878ED
:100C90003A25326868783A25326868783A253268A9
:100CA00068783A253268687800253032783A2530FD
:100CB00032783A253032783A253032783A25303257
:100CC000783A25303278003078255800257520256F
:100CD0007520257800307825580025752025750069
:100CE000307825303258002575202575202578006C
:100CF000307825303258002575202575202578005C
:100D00003078253032580025752025780030782538
:100D1000303258002575202575003078253032583E
:100D2000002575202575003078253032580025754E
:100D30000064657465637465642061743A2030787A
:100D40002578202825642900253032753A2530344D
:100D5000583A253034583A253032580A006F6666C2
:100D6000006F6E006C6566740072696768740025B8
:100D70007520257500257520257820257820257873
:100D800020257820257820257820257820257800B2
:100D900025752025750025333273256320256C6465
:100DA0000053442F4D4D43206261636B656E642098
:100DB0006E6F7420617661696C61626C652E00648F
:100DC00020006675736500686F73746E616D6500F1
:100DD0007265736574007764726573657400696F1A
:100DE0000061646320676574006D61630069726D02
:100DF000702072656365697665006C636420636C5E
:100E0000656172006C6364207772697465006C635D
:100E10006420676F746F006C6364206368617200A4
:100E20006C6364207265696E6974006C636420731E
:100E300068696674006C6364206261636B6C6967E7
:100E4000687400736420646972007364206D6B645D
:100E50006972006E65746D61736B0069700067770D
:100E600000693263206465746563740069326320CD
:100E700072626200693263207262640069326320C8
:100E8000727764006932632077626200693263209E
:100E90007762640069326320777764007063663834
:100EA0003537347820726561640070636638353791
:100EB0003478207365740068656C700076657273B1
:100EC000696F6E00656570726F6D207265696E691D
:100ED0007400BF0D220BC20D8E0BC70DCC0BD00DB5
:100EE000EA0BD60DFA0BDE0DAA3CE10D8B3DE90DA8
:100EF000373EED0D1842FA0DB143040E9B430E0E22
:100F00004F43170EE842200EA7422B0E8042350EAB
:100F10005A42430EEB434A0EDB43530EAF445B0E83
:100F2000F4445E0E6A44610ECE416C0E7641740E3E
:100F300012417C0EAE40840E4A408C0EE13F940E6E
:100F4000773F9C0E123FAA0EA83EB70EE733BC0EA9
:100F50003734C40EE23300000000443A2073645F6B
:100F600070696E67206661696C65642C20656565D3
:100F70006B2E2020636172642072656D6F766564EC
:100F80003F0A006364696E6F70737578585B000088
:100F900014BE88E10FB6F894809360001092600050
:100FA0000FBE10926E0010926F001092700011240C
:100FB0001FBECFEFD0E1DEBFCDBF11E0A0E0B1E0BA
:100FC000EEE0F0EA02C005900D92A433B107D9F724
:100FD00018E0A4E3B1E001C01D92AE32B107E1F721
:100FE00003D00C94F3470CC8CF93DF9382E081B910
:100FF00088EB84B984E58AB902D200D08DEC90E008
:10100000ADB7BEB712969C938E9311970E94484934
:10101000789486EB90E0EDB7FEB7928381830E94CF
:10102000484988E10FB6F894809360001092600000
:101030000FBE86E880937A0010927C000F900F908C
:1010400027D20E94C74582E7B5D400D000D0EDB7C3
:10105000FEB731962BE930E0ADB7BEB712963C93A0
:101060002E931197828313820E944849EDB7FEB7F1
:101070003A970FB6F894FEBF0FBEEDBF319680E8E9
:1010800090E0ADB7BEB712969C938E931197809166
:10109000480482831382809149048483158280915D
:1010A0004A048683178280914B0480871186809141
:1010B0004C048287138680914D04848715860E9494
:1010C0004849EDB7FEB73E960FB6F894FEBF0FBE87
:1010D000EDBF0E943945C0E0D0E00E94BE4580913E
:1010E000440490914504892B31F40E9414238823F1
:1010F00011F40E94272980913D0482FF0DC0F894CD
:1011000028E088E190E00FB6F894A89580936000FD
:101110000FBE20936000FFCF81FFDFCFF894FE0168
:101120000995DBCF1F93CF93DF9310E0C0E0D0E0B1
:10113000CE010E94514E182788E09CE810FB1695BE
:101140000EF419278A95D1F72196C231D10581F77E
:10115000812FDF91CF911F910895EF92FF920F930E
:101160001F93CF93DF938B01EA01040F151F7C01BE
:10117000E40EF51E06C02197C701F80160810E94A8
:10118000594E015010400894E108F108209799F752
:10119000CDB7DEB7E6E00C94F04FABE0B0E0E3EDA6
:1011A000F8E00C94D44F8E010A5F1F4FC8016EEE19
:1011B00070E046E050E00E940B4880E090E0B8010B
:1011C00046E050E0CADF80ECE82E88EAF82EFB8289
:1011D000EA8280E09AE59D838C838E010E5F1F4F2B
:1011E00086E090E0B80144E050E0B7DFFB82EA829D
:1011F00080E092E09D838C838EE090E0B80144E033
:1012000050E0ABDF8FEF9FEF9B838A838FEF90E0FF
:101210009D838C838AE090E0B80144E050E09DDF3C
:1012200081DF898382E190E0BE016F5F7F4F41E003
:1012300050E093DF2B96E6E00C94F04FA1E0B0E095
:10124000E4E2F9E00C94D74F0E94E8296BDF182FF5
:10125000CE01019662E170E041E050E00E94414E13
:101260008981181709F099DFCDD20E94C345FBD3BD
:101270000E94CC332196E3E00C94F34F0895089537
:101280001F93182F8A3019F48DE0FADF03C08B31D9
:1012900009F41EE58091C00085FFFCCF1093C600C5
:1012A00080E090E01F910895A0E0B0E0EAE5F9E069
:1012B0000C94D24F8091C00087FF9CC01091C60053
:1012C0001A3019F01D3009F063C088E290E00E94E6
:1012D000D545EC01009769F400D081E291E0ADB70B
:1012E000BEB712969C938E9311970E9448490F9017
:1012F0000F90E0911701F0911801108200D08FE15A
:1013000091E0EDB7FEB7928381830E9448490F9028
:101310000F909BE1C92E91E0D92E86EFE82E8FEF3A
:10132000F82E84E391E0BE0148E250E00E945F3471
:101330008C0109960997F0F0FFEF073F1F0714F0A3
:10134000F80103C0F701E01BF10BEC0FFD1F108249
:1013500000D000D0ADB7BEB71296DC92CE921197F6
:101360001496DC93CE9313970E9448490F900F90E8
:101370000F900F90BFEF073F1B079CF2CE010E941A
:10138000824684E391E0909318018093170132C064
:101390006091280870912908812F72DFE091170170
:1013A000F0911801183039F481E0E433F80711F1B5
:1013B00008F1319705C0A1E0EF36FA0730F4119338
:1013C000F0931801E093170115C000D000D0EDB7DD
:1013D000FEB7319685EF90E0ADB7BEB712969C93FD
:1013E0008E931197128313820E9448490F900F9099
:1013F0000F900F90CDB7DEB7E8E00C94EE4F9FB79B
:10140000F8941092C50087E68093C40086E080932C
:10141000C200A1ECB0E08C9188698C93E0ECF0E024
:1014200080818D7F80839FBF8C918F778C9380E4A8
:1014300099E060E070E00C94A9488CE08093810012
:1014400081EE94E09093890080938800EFE6F0E0CD
:1014500080818260808308951F920F920FB60F9251
:1014600011248F939F9381E08093210890913E04F3
:10147000892F8F5F80933E04823318F091539093AD
:101480003E049F918F910F900FBE0F901F90189563
:101490002C9A2B9A80E58CBD81E08DBD08958EBD80
:1014A00088EC01C081500DB407FC03C08823D1F73C
:1014B00002C0882359F400D086E391E0EDB7FEB76F
:1014C000928381830E9448490F900F908EB50895B2
:1014D0005E9A08958BB190E489278BB90895A2E1B3
:1014E000B0E0E5E7FAE00C94D04F182F7B015901EA
:1014F0006A01FB01608182E1689FB0011124695A91
:101500007E4FCE01019642E150E00E940B4811232C
:1015100051F4EB85FC853097C9F0C701B601A501F0
:10152000202F099514C0113049F4ED85FE853097C0
:1015300069F0C701B601A501099509C0123031F45F
:10154000ED81FE81309711F0C701099580E0629628
:10155000EAE00C94EC4F6F927F929F92AF92BF9211
:10156000CF92DF92EF92FF920F931F93DF93CF936F
:10157000CDB7DEB762970FB6F894DEBF0FBECDBF12
:10158000982E7B013A0158016901FB01608182E1DB
:10159000689FB0011124695A7E4FCE01019642E145
:1015A00050E00E940B48992019F4EF81F88505C09E
:1015B000F1E09F1651F4E985FA85309791F0C70163
:1015C000B301A6019501099509C082E0981649F476
:1015D000E989FA89309729F0C70109959B01AC0187
:1015E00004C020E030E040E050E0B901CA0162965A
:1015F0000FB6F894DEBF0FBECDBFCF91DF911F9124
:101600000F91FF90EF90DF90CF90BF90AF909F90A1
:101610007F906F900895A2E1B0E0E1E1FBE00C94CF
:10162000D64F8C01CE01019667E571E042E150E0B2
:101630000E940B48EB81FC81C80109956296E4E0A9
:101640000C94F24FA2E0B0E0E8E2FBE00C94D04F43
:10165000DC015B0101C011968C918032E1F300D076
:1016600000D000D02DB73EB72F5F3F4FEDB7FEB78C
:10167000B283A1838EE691E0F90193838283CE0148
:101680000196958384830E94E8492DB73EB72A5F6F
:101690003F4F0FB6F8943EBF0FBE2DBF019719F014
:1016A0002FEF3FEF36C0E980FA8000E010E039E626
:1016B000C32E31E0D32E00D000D000D0ADB7BEB7DE
:1016C0001196C801880F991F8A0D9B1DEDB7FEB7B3
:1016D000928381831396DC92CE921297F801EE0DDD
:1016E000FF1D808114968C93149715961C920E946E
:1016F000C7490F5F1F4F2DB73EB72A5F3F4F0FB649
:10170000F8943EBF0FBE2DBF00311105A1F620E2B7
:1017100030E0C9012296EAE00C94EC4FCF93DF93BE
:1017200089E087BFE0E0F0E0B49187BFE3E0F0E05C
:10173000A49187BFE2E0F0E0349187BFE1E0F0E000
:1017400024918DB79EB70E970FB6F8949EBF0FBE2B
:101750008DBFEDB7FEB73196CDB7DEB77A8369831B
:101760005383428381E791E095838483B683178214
:10177000A087118632871386248715860E9499498F
:101780002DB73EB7225F3F4F0FB6F8943EBF0FBE56
:101790002DBFDF91CF91089500D000D000D0EDB7DC
:1017A000FEB73196ADB7BEB712967C936E93119784
:1017B0005383428383E991E0958384830E9499490E
:1017C0002DB73EB72A5F3F4F0FB6F8943EBF0FBE0E
:1017D0002DBF0895FC018081882319F02FEF3FEF82
:1017E00007C080913D04826080933D0420E030E09A
:1017F000C901089580913D04846080933D0480E098
:1018000090E00895A4E0B0E0E8E0FCE00C94D64F4E
:1018100088E494E060E070E046E050E00E94414ED1
:101820008E010F5F1F4FC80166E070E044E050E09A
:101830000E94414E89819A819093260680932506C5
:101840008B819C819093280680932706C8016AE0CB
:1018500070E044E050E00E94414E89819A8190936B
:101860002206809321068B819C819093240680938D
:101870002306C8016EE070E044E050E00E94414E53
:1018800089819A8190931E0680931D068B819C818D
:101890009093200680931F062496E4E00C94F24F68
:1018A0002C988FEFFCDD80E49FE10197F1F72C9AF3
:1018B0000895FF920F931F93182FF62E042F282FB1
:1018C00030E0C9018F7190704B977CF420763070B6
:1018D00085E0359527958A95E1F78091710190E033
:1018E0002817390711F0822F0CD02C981F71802FE8
:1018F000812BD5DD8F2DD3DD2C9A1F910F91FF9079
:1019000008951F93182F8FE163E040EAD2DF612F23
:1019100063708FE140E8CDDF109371011F9108954E
:101920001F93182F2C988AE7BADD812FB8DD2C9AE7
:101930001F9108950F931F93182F062F282F30E023
:10194000C9018F7190704B977CF42076307095E0D0
:10195000359527959A95E1F78091710190E02817C8
:10196000390711F0822FCDDF2C981F71812F8064F1
:1019700096DD802F94DD2C9A1F910F9108951F936F
:10198000682F192F82E0D6DF83E0612FD3DF1F910C
:1019900008951F93682F192F80E0CCDF81E0612F1D
:1019A000C9DF1F9108952C988AE379DD80E077DD07
:1019B0002C9A08951F93182F282F30E0C9018F719A
:1019C00090704B977CF42076307045E035952795E4
:1019D0004A95E1F78091710190E02817390711F0DD
:1019E000822F8FDF2C98812F8F7159DD80E057DD9A
:1019F00017FF02C080E053DD2C9A1F9108950F93CA
:101A00001F93982F162F072F84ED692F93DF86EDF4
:101A1000612F90DF87ED602F8DDF8AEECBDF80FDB9
:101A2000FCCF1F910F9108950F931F93682F84EDA2
:101A300081DF82ED61E040E83CDF8AEEBBDF80FDC4
:101A4000FCCF82ED61E040EA34DF88EDB3DF082FA0
:101A500089EDB0DF382F20E010E0022B132BC801F6
:101A60001F910F9108958FEF8093740119DF88E023
:101A700060E060DF89E060E05DDF8AE06FEF5ADF01
:101A80008BE06FE057DF84E060E054DF85E060E1E9
:101A900051DF8CE060E04EDF8DE060E04BDF8EE0F8
:101AA00060E048DF8FE060E045DF10924004109274
:101AB0003F0481EC60E840EAFCDE80EC6DE040E849
:101AC000F8DE82EC62E340E8F4DE80E060E070E0A3
:101AD00096DF80E0A9DF90FF07C082EC61E040E87C
:101AE000E8DE84EC62E106C082EC61E040EAE1DE1F
:101AF00084EC65E11FDF86EC62E11CDF87EC6CE0C3
:101B000019DF8AEC68EF16DF8BEC61E013DF84EEFF
:101B1000609148040FDF85EE609149040BDF82EE8F
:101B200060914A0407DF83EE60914B0403DF80EE8F
:101B300060914C04FFDE81EE60914D04FBDE88E392
:101B400063E8F8DE84E162E17CE059DF8BE16BED74
:101B5000F1DE82E162E170E052DF8FE164E040E8B3
:101B6000A8DE8EE160E840E8A4DE109274010895DA
:101B7000809174018823A9F482EC1CDF8273823384
:101B800031F0809172018F5F809372016CDF80EC85
:101B900011DF8D3031F0809173018F5F809373017D
:101BA00062CF0895A4E0B0E0E8EDFDE00C94D24FE0
:101BB00089E300DF882309F497C080913F04909166
:101BC0004004E7DEF0DE082FEEDE382F20E010E0E4
:101BD000202B312B3093400420933F047E01089446
:101BE000E11CF11CE0DE898387010F5F1F4FDBDE04
:101BF000F7018183D8DEF8018183D5DE0F5F1F4FA7
:101C0000F801818389819A812CEFE22E2FEFF22E49
:101C1000E80EF91E4297875E914030F409E216E023
:101C20006801CE0CDF1C16C000D000D08FE991E017
:101C3000EDB7FEB792838183F482E3820E94484924
:101C40000F900F900F900F900EDF4EC0ACDEF8019A
:101C500081938F010C151D05C9F7F0924704E0929E
:101C600046049091350680913606F8E080309F0753
:101C700061F086509840B9F40E94ED31809146049D
:101C800090914704892B79F00DC00E94C33181E007
:101C90000E943F2A8091460490914704892B19F0B5
:101CA0000E948B32A4D060913F0470914004CB011C
:101CB00001978050904130F08CE06FEF3BDE8DE07B
:101CC0006FE00DC061508CE035DE60913F04709193
:101CD000400461507040672F770F770B8DE02ADE4C
:101CE0008EE160E440E8E5DD2496E8E00C94EE4FF8
:101CF0001F9389E35FDE882309F477C08CE15ADE05
:101D0000182F8BE160E840EAD4DD14FF1DC083E1A9
:101D10008BDE81E189DE92FF0BC000D084E492E08B
:101D2000EDB7FEB7928381830E9448495C9A0AC04E
:101D300000D082E392E0EDB7FEB7928381830E94E8
:101D400048495C980F900F9013FF17C08DE132DE69
:101D500081FF0BC000D082E192E0EDB7FEB7928325
:101D600081830E9448490F900F908CE168E040EA1F
:101D7000A0DD8DE16AE040EA9CDD9FB7F894809198
:101D8000F405882311F081E004C088E08093F40515
:101D900080E09FBF882349F505DF1092F40510FF0E
:101DA0000FC000D08AEF91E0EDB7FEB79283818338
:101DB0000E9448490F900F908CE161E040EA79DD84
:101DC00011FF0FC000D081EE91E0EDB7FEB7928316
:101DD00081830E9448490F900F908CE162E040EAB5
:101DE00068DD8BE160E840E864DD1F9108951F9392
:101DF000CF93DF9314E68FE1DDDD83FD03C0112374
:101E000021F00FC01150B8F70CC000D087E592E068
:101E1000EDB7FEB7928381830E9448490F900F90DF
:101E200034C084E060E086DD85E060E183DD86E04B
:101E3000609146047FDD2091460430914704205094
:101E4000304F87E0632F76DD80E090E198DD80E021
:101E500067DDC0E0D0E006C0FE01E75DF94F80819C
:101E60005FDD21968091460490914704C817D907F9
:101E700098F38FE160E840E81CDD8FE160E840EA1C
:101E800018DD8FE168E040E814DDDF91CF911F910C
:101E900008951092B9008CE08093B800419A409A5E
:101EA00008958093BC008091BC0087FFFCCF809197
:101EB000B900887F089584E98093BC008091BC00BC
:101EC00084FFFCCF1092BC000895982F84E8809383
:101ED000BC0084EA8093BC008091BC0087FFFCCFEB
:101EE0008091B900887F883011F08031D9F4990F42
:101EF000962B9093BB0084E88093BC008091BC003B
:101F000087FFFCCF9091B900987F662321F480E091
:101F1000983149F405C0613029F480E0903419F417
:101F200081E0089580E00895FF920F931F93062F9C
:101F3000182F84E9F82E19C0812F60E0C6DF8823AE
:101F400059F084E98093BC008091BC0084FFFCCFF1
:101F50001092BC00812F0CC0F092BC008091BC009C
:101F600084FFFCCF1092BC001F5F101728F38FEF87
:101F70001F910F91FF900895FF920F931F93CF939E
:101F8000DF93162F042FF52E60E09FDF8823B9F032
:101F90001093BB0084EC85DF883289F4F092BB009B
:101FA00084EC7FDF883259F40093BB0084EC79DF46
:101FB000883229F4802F9F2D9C01E90102C0CFEFC8
:101FC000DFEF79DFCE01CDB7DEB7E5E00C94F14F5E
:101FD0000F931F93CF93DF93162F042F60E075DFCD
:101FE000882379F01093BB0084EC5BDF883249F4DE
:101FF0000093BB0084EC55DF883219F4C02FD0E089
:1020000002C0CFEFDFEF57DFCE01DF91CF911F91FD
:102010000F9108951F93CF93DF93162F60E055DF44
:10202000882349F01093BB0084EC3BDF883219F41D
:10203000C12FD0E002C0CFEFDFEF3DDFCE01DF9157
:10204000CF911F9108950F931F93CF93DF93182F74
:10205000062F60E03ADF882329F10093BB0084EC6F
:1020600020DF8832F9F484EA1CDF8031D9F4110FC3
:1020700011601093BB0084E814DF803499F484EC81
:1020800010DF803579F41091BB0084EC0ADF8035D5
:1020900049F42091BB00912F80E0C22FD0E0C82BE3
:1020A000D92B02C0CFEFDFEF06DFCE01DF91CF915A
:1020B0001F910F9108950F931F93182F062F60E023
:1020C00004DF8823C9F00093BB0084ECEADE883289
:1020D00099F484EAE6DE803179F4110F11601093EF
:1020E000BB0084E8DEDE803439F484ECDADE80354F
:1020F00019F41091BB0001C01FEFDDDE812F1F918D
:102100000F9108951F9361E0E0DE882369F084EC6D
:10211000C8DE803549F41091BB0084E8C2DE883502
:1021200019F48091BB0001C01FEFC5DE812F1F9104
:1021300008951F93162F60E0C8DE1093BB0084E85B
:10214000B0DEB9DE8FEF9FEF1F9108951F9361E01E
:10215000BCDE882369F084ECA4DE803549F410915C
:10216000BB0084E89EDE883519F48091BB0001C075
:102170001FEFA1DE812F1F910895FC018091930133
:10218000882309F443C080919401823021F0873084
:1021900009F03DC02EC020919701309198018091A7
:1021A000970190919801232F3327809590959070F7
:1021B00028173907A1F080919501909196018E5EC4
:1021C000974809F58BE08093940180919701909155
:1021D0009801892F9927909396018093950180917A
:1021E0009701909198019070909398018093970136
:1021F0000EC080919501909196018F7D90939601EC
:102200008093950104C080E010929301089580911D
:1022100094018083809195019091960192838183AE
:102220008091970190919801948383838091990183
:102230008583109298011092970110929601109246
:1022400095011092990181E0DFCF982F6091810173
:10225000662339F4809182018F3019F490938001C4
:1022600055C070918B01671738F180918C01681708
:1022700018F580919101292F30E040919A015091F9
:102280009B01882381F0862F90E0871B910902C073
:10229000220F331F8A95E2F7422B532B50939B0159
:1022A00040939A0133C0440F551F242B352B309394
:1022B0009B0120939A012AC070918D01671730F11C
:1022C00080918E01681710F580919101292F30E0DF
:1022D00040919C0150919D01882381F0862F90E0D0
:1022E000871B910902C0220F331F8A95E2F7422B08
:1022F000532B50939D0140939C0108C0440F551FE0
:10230000242B352B30939D0120939C016F5F6093AC
:102310008101089520982898529A5A9885B58A7F05
:1023200085BD85B5826085BD87EC87BD16BCEEE6B0
:10233000F0E08081826080830895AC0190919E01DD
:1023400080919F01981711F480E00895892F8F5F85
:10235000877080939E0190E0FC01EE0FFF1FE80F55
:10236000F91FEE0FFF1FDA01E056FE4F86E00190E5
:102370000D928150E1F781E00895282F809193011B
:10238000882309F0D7C280917F01882381F590913D
:102390007C01222321F49F5F90937C01CBC299237F
:1023A000B9F091E090937F0190937D0110927E01AE
:1023B00010929D0110929C0110929B0110929A0123
:1023C0008FEF8093810190937B0110927701B2C2CD
:1023D0008091790190917A012FEF8F3F920709F454
:1023E000A9C2019690937A0180937901A3C280914A
:1023F0007D01882309F491C0222349F080917B015B
:102400008F5F80937B018C3908F4D5C145C1209141
:102410007C01822F8E53893380F480917B018E3131
:1024200028F08C3328F46EE872E03CC08F3028F03E
:102430008F3118F46FE972E035C0822F87508530F4
:1024400018F087508930C8F490917B01892F87500C
:10245000853018F08750893080F460EB72E09093FB
:1024600076012C502B3018F09C509B3098F4109231
:10247000750180E48093770115C02350253070F4F6
:1024800080917B01863150F0823240F461EC72E041
:102490008093760181E08093750104C010927F01E2
:1024A00060E070E080917F01882331F082E891E064
:1024B00041E150E00E940B4810928101809192010D
:1024C000482F50E080FF21C0809182018731E9F0E0
:1024D0008930D9F020917B0180918401821760F4CA
:1024E00030E090E0880F991F821793072CF05695E3
:1024F0004795842F809507C080917501882329F422
:1025000056954795842F8170A0DE81E080937C01F1
:1025100010927B0110927D014EC180917E01882333
:1025200009F43CC1222309F4BEC05091810160919D
:102530008F015617B9F480919001813099F4809100
:10254000920180FD0CC090917C01809187019817C9
:1025500008F4A2C080918801891708F49DC01092E8
:10256000900129C140917B014F5F40937B01809195
:1025700082018F3009F05FC080919001882309F0BB
:102580005AC04A3118F1563009F581E08093900124
:1025900088E18093820187E080938F0110928B0104
:1025A00010928C0110928D0180938E0120919C01DC
:1025B00030919D01220F331F8091800190E0822B8A
:1025C000932B90939D0180939C016DC0242F30E04C
:1025D0008091860190E0880F991F2817390734F001
:1025E000583020F08AE080938F013FC05A3008F4C1
:1025F000E2C080E18093820199E090938B0181E1B8
:1026000080938C0181E080938D0190938E012091C5
:102610009C0130919D01C90180709370892B09F450
:10262000CAC030939A0110929B01307030939D0183
:1026300020939C01C0C08091920180FF1AC0242F7A
:1026400030E08091860190E0880F991F28173907A4
:1026500084F0252F30E0862F90E002972817390765
:1026600044F080919001882321F481E080939001CF
:102670001AC04C3908F49FC0252F30E0862F90E017
:1026800001972817390741F480919001882321F49C
:102690005F5F509381018FC010927F0110927C0187
:1026A00010927B0188C080919201282F30E0909198
:1026B0007C0180FF42C0809184018917B0F4369577
:1026C0002795822F80958170C0DD8091920190E0E6
:1026D000969587958170B9DD8091920190E09695ED
:1026E000879581708093750123C08091830198172D
:1026F000D8F02091760180918601821780F430E035
:1027000090E0880F991F821793074CF090E080911A
:102710007501882309F491E09093750102C09091AE
:102720007501892F92DD04C010927F0110927B0108
:1027300080917B018093760114C08091830198176A
:1027400098F080918401891778F020917B01809125
:102750008501281748F080918601821728F081E0D2
:1027600074DD10927E0118C080918701981780F067
:1027700080918801891760F090917B018091890197
:10278000981730F080918A01891710F080E0E8CF27
:1027900010927F0110927B0181E005C0222331F469
:1027A00080917C018F5F80937C0105C081E08093E4
:1027B0007E0180937B0180917F01882309F4BAC058
:1027C0003091810180918F01381709F0B3C0809159
:1027D0009001882309F0AEC06091190170911A012F
:1027E00040919C0150919D016417750769F4809197
:1027F000790190917A018052934030F48091780170
:102800008F5F8093780102C01092780181E08093FD
:102810009301209182012F3031F44F5F514031F507
:10282000109293014BC0223009F53323F9F48091C3
:10283000790190917A01805B9440B0F480911B0102
:1028400090911C0190939B0180939A0170939D013C
:1028500060939C018091990181608093990110920D
:102860007A011092790102C0109293012093940191
:1028700080919A0190919B0190939601809395018C
:10288000223029F490931C0180931B010FC0273044
:1028900069F42091770130E080919C0190919D0135
:1028A000822B932B90939D0180939C0180919C019E
:1028B00090919D019093980180939701809193014D
:1028C000882371F140919C0150919D016417750717
:1028D000B9F420911B0130911C0180919A019091D3
:1028E0009B012817390761F48091790190917A0151
:1028F0008C5D954028F480919901816080939901C5
:1029000080919A0190919B0190931C0180931B01EF
:1029100050931A014093190110927A011092790193
:1029200010927F0110929D0110929C0110927C01E7
:1029300010927B018091930108951F920F920FB620
:102940000F9211241F932F933F934F935F936F9395
:102950007F938F939F93AF93BF93EF93FF9387B52D
:10296000885387BD83B1982F917080FD02C05A9A19
:1029700001C05A98892F01DD882399F010919F0199
:102980001F5F177080919E01181759F086E0189FFD
:10299000C001112480569E4FF0DB882311F0109364
:1029A0009F01FF91EF91BF91AF919F918F917F9187
:1029B0006F915F914F913F912F911F910F900FBE9B
:1029C0000F901F9018958295807F860F8093D0017D
:1029D0000895FF920F931F93182FF62E42D1082FC0
:1029E000812F6F2D3ED10295007F802B1F910F917B
:1029F000FF900895FF920F931F93182F062FF42E28
:102A000062956F7043D10F70812F602F4F2D3ED193
:102A100018EC05E380E06F2DDCDF902F9A95F1F73D
:102A2000115087FF03C01123A9F702C0112359F4E5
:102A300000D082ED92E0EDB7FEB7928381830E94D1
:102A400048490F900F901F910F91FF9008951F9389
:102A5000CF93DF93182FEB018A3091F403C080E20B
:102A6000BE01F5DF2091D001822F90E08F70907031
:102A7000892BA9F7203470F120542093D0012AC06B
:102A80006091D0018D3021F4607F6093D00122C02D
:102A9000603110F460580DC0603210F4605509C008
:102AA000603310F4605905C0603410F060E001C07C
:102AB0006056606880E041E09DDF81E0612F41E089
:102AC00099DF8091D0018F5F8093D001803411F421
:102AD0001092D00180E090E0DF91CF911F91089596
:102AE0006C60982F990F962B80E0692F83CFFF920F
:102AF0000F931F93CF93DF93982F8B01F42E883081
:102B0000A0F4990F990F990F906480E0692F72DFFC
:102B1000C0E0D0E0F801EC0FFD1F81E060814F2D97
:102B200069DF2196C830D105A9F7CDB7DEB7E5E05A
:102B30000C94F14F462F882311F468E101C06CE139
:102B400080E058CF80E061E041E054CF0F931F93C5
:102B500048D080E991E020E931E0F9013197F1F7BF
:102B60000197D9F780E063E041E090D080E89EE3F0
:102B70000197F1F780E061E048D000EA1FE0C8016A
:102B80000197F1F780E061E040D0C8010197F1F7CB
:102B900080E062E041E07AD0C8010197F1F780E07F
:102BA00068E241E027DF80E060E041E099DF81E01A
:102BB00090E0C8DF80E066E041E01CDF80E060E894
:102BC00041E018DF87E295E160E070E00E94A948EB
:102BD00090934204809341041092D0011F910F9171
:102BE00008951092430480E260E0A3CA8093D1016B
:102BF00090914304882311F0906801C09F779093CF
:102C0000430480E26091430494CA1F93882399F09F
:102C1000609143046F6080E28CDA60914304862FF8
:102C20008064809343046F6480E283DA80E28EDA0A
:102C3000182F1F700CC080E2609143047ADA609113
:102C4000430460646093430480E273DA10E06091AF
:102C500043046F7B6093430480E26BDA812F1F9102
:102C6000089590914304292F2062882321F09063D6
:102C70009093430403C02F7E2093430481E0C5DF7B
:102C8000909143049F7D909343040895609343047F
:102C9000882319F060616093430490914304292FC5
:102CA0002F7D8091D101882321F020682093430457
:102CB00003C09F759093430480E061E0A6CFA2E03B
:102CC000B0E0E5E6F6E10C94D84FDC01009781F125
:102CD0006230710568F1ED91FC911197660F771FD5
:102CE00080E090E016962D913D914D915C91199761
:102CF000620F731F841F951F0190F081E02DAE01BC
:102D00004F5F5F4F22E030E00995882389F02981E9
:102D10003A812115310571F08FEF273F380741F0D7
:102D2000C9014096079720F08FEF283F380710F031
:102D300020E030E0C9012296E2E00C94F44FA2E0DA
:102D4000B0E0E5EAF6E10C94CA4F5C01009709F4A3
:102D500049C06230710508F445C0DC0116966D90DB
:102D60007D908D909C9019972E010894411C511CC8
:102D7000660F771F7B0100E010E0E60CF71C081DD2
:102D8000191DD501ED91FC910190F081E02DC80154
:102D9000B701A20122E030E00995882319F1C9802A
:102DA000DA80C114D10401F1C60140960897D0F031
:102DB000B8EFCB16BFEFDB0610F0CC24DD241A826F
:102DC0001982D501ED91FC910480F581E02DC801B7
:102DD000B701A20122E030E00995B601C114D10487
:102DE00039F602C080E001C081E02296E0E10C9457
:102DF000E64FAAE0B0E0EFEFF6E10C94C84F3C01DB
:102E00002B01009709F48FC0DC01ED91FC91119723
:102E1000208131813A8729872480358016968D91CB
:102E20009D910D90BC91A02D8D839E83AF83B8871B
:102E3000F30182859385A485B585B695A795979569
:102E400087959C838B834A01CC24DD2442E0A42E09
:102E5000B12C41C0C501880F991F7C0100E010E032
:102E60002D813E814F815885E20EF31E041F151FF0
:102E7000C801B701AE014F5F5F4F22E030E0A98586
:102E8000BA85FD010995882309F44DC089819A818D
:102E9000892BF1F4C114D10429F4EFEFFFEFFA8389
:102EA000E98302C0DA82C982C801B701AE014F5F6F
:102EB0005F4F22E030E0F1010995882391F00894FA
:102EC000810891088114910411F465010DC0650118
:102ED0000894A11CB11C2B813C81A216B30608F4F6
:102EE000B9CF81149104E1F432E043165104E8F0C3
:102EF000DA82C982440C551CB20180E090E02D8139
:102F00003E814F815885620F731F841F951FAE014C
:102F10004F5F5F4F22E030E0F1010995882329F4EB
:102F2000C301B6010CDFCC24DD24C6012A96E2E100
:102F30000C94E44F80E190E00895AAE0B0E0E3EA69
:102F4000F7E10C94C84F2C017A8369835C834B832F
:102F5000009709F407C1672B09F404C1452B09F454
:102F600001C1DC019D96AD90BD90CD90DC90D097D5
:102F700095962D913D914D915C919897EB81FC81B7
:102F8000CF01A0E0B0E08A0D9B1DAC1DBD1D281730
:102F900039074A075B0740F4B9016A197B097C834A
:102FA0006B83672B09F4E1C0D201ED91FC9111977D
:102FB00020883188D196ED91FC91D297FA87E987E4
:102FC000EF2BE9F593962D913C9194973A872987B9
:102FD000232B39F4A114B104C104D10409F4C5C0F0
:102FE000C1C0A114B104C104D10449F18601750125
:102FF00031018824992466277727CB016619770940
:10300000880999096D837E838F83988713C0D201C5
:103010008D919C9169857A8552DE9A878987892B63
:1030200009F4A0C06D817E818F819885E60EF71E20
:10303000081F191FE614F7040805190540F708943E
:1030400021083108A220B3200894211C311CCB8018
:10305000DC80D201ED90FC90E114F10409F1E985E6
:10306000FA85E230F105E0F03297BF0180E090E0B0
:103070003296FA87E987D70150962D913C91519766
:1030800040E050E00E94604F9B01AC01F701828953
:103090009389A489B589280F391F4A1F5B1F04C073
:1030A00020E030E040E050E081010A191B09C01621
:1030B000D10608F48601D701ED91FC91C501A0E08D
:1030C000B0E0280F391F4A1F5B1F0190F081E02DEF
:1030D000CA01B90149815A8198010995882339F1BA
:1030E000C01AD10AC801A0E0B0E0F20125A536A5BA
:1030F00047A550A9280F391F4A1F5B1FD2019D9673
:103100002D933D934D935C93D097C8018A0D9B1DE1
:103110008215930598F08D919C9169857A85CFDD14
:103120009A878987892B41F4F20112AA11AA4B814F
:103130005C814C195D091BC0AA24BB24E985FA8572
:10314000D201D296FC93EE93D197C114D10439F0F9
:1031500029813A81200F311F3A8329837ACF4B810D
:103160005C8105C04FEF5FEF02C040E050E0CA0154
:103170002A96E2E10C94E44FFC01009711F480E000
:10318000089583A194A196A785A710AA17A681E008
:103190000895ADE0B0E0EFECF8E10C94D24F8C0173
:1031A0006A017B01B901D9014D915C911197129689
:1031B0008D919C911397809613969C938E93129762
:1031C000F8018081853E09F4C7C0882309F4C4C092
:1031D000FA0187A190A5A1A5B2A50097A105B10507
:1031E00039F4DA019796CD92DD92ED92FC929A979E
:1031F0004115510509F4B2C00115110509F4AEC01D
:10320000F8019081992309F4A9C083858F30A9F52D
:10321000892F90E08F73907001972DE030E0829FAE
:10322000B001839F700D929F700D1124DE011196E5
:10323000EDE1F1E08DE001900D928150E1F7DA01CE
:10324000A60FB71F20E030E0AE014F5F5F4F0FC009
:10325000FA01E20FF31F8081F801E80FF11D808170
:103260008D932F5F3F4F2D30310509F475C0C90193
:10327000860F971F4F9760F36FC0DA018C918823F8
:1032800009F050C07801680120E0F6019081903289
:10329000A1F09C93F801848583FF08C0F60180812A
:1032A000813420F08B3510F4905E9C932F5F08944E
:1032B000C11CD11C1196283041F7DA018C91853060
:1032C00011F485EE8C93F8018085803211F4322F51
:1032D00025C0FA01E20FF11D8EE28083322F3F5F9D
:1032E0002C5FD70118969C919032C1F0FA01E30F40
:1032F000F11D9083D8011C968C9184FF09C0D701E1
:1033000018968C91813420F08B3510F4905E908368
:103310003F5F0894E11CF11C321719F7FA01E30F23
:10332000F11D1082F8018385DA0190968C939097B5
:10333000828D938D92969C938E939197848D958D8B
:10334000A68DB78DFA0183A394A3A5A3B6A381E0AC
:10335000DB0114968C9302C081E001C080E02D96C1
:10336000E8E00C94EE4FA0E1B0E0E9EBF9E10C9459
:10337000D24F8C016230710510F480E035C00097A7
:1033800029F440E050E060E070E016C06250704008
:1033900080E090E0F8012089318940E050E00E940F
:1033A000604FAB01BC01F80182899389A489B5897A
:1033B000480F591F6A1F7B1FDE01119680E1FD0136
:1033C00011928A95E9F7F8018081918120893189EC
:1033D000FC01C680D780CB01BA01AD010AE917E133
:1033E000EE24FF24F60109956096E8E00C94EE4F78
:1033F000A7E2B0E0EEEFF9E10C94C84F2C017FA3F7
:103400006EA3009709F4B0C06115710509F4ACC052
:10341000DC018D909C901197F401208831889D9655
:10342000AD90BC909E979F966D907C90D0978BE2CC
:10343000DB011D928A95E9F7FE01319685E0DF01F7
:103440001D928A95E9F7A114B10409F075C0F40141
:103450002288338886899789281A390A6DC07301B2
:1034600000E010E0A114B10441F4D40156966D912E
:103470007D918D919C9159972DC08114910421F1DA
:10348000B2E0AB16B10400F1EEEFFFEFAE0EBF1EDF
:10349000B50180E090E022E030E0A20EB31ED4013E
:1034A00050962D913C91519740E050E00E94604F22
:1034B0009B01AC01F40182899389A489B589280F05
:1034C000391F4A1F5B1F04C020E030E040E050E09D
:1034D000CA01B9016E0D7F1D801F911F1C821B82C6
:1034E000D401ED91FC918101061917090280F38145
:1034F000E02DAE014A5F5F4F20E230E0A9ECEA2EFA
:10350000A8E1FA2E6E010894C11CD11C09958823EC
:1035100059F18B819C81680E791E6214730480F0CE
:10352000C401B501CCDB5C0166247724009741F42B
:10353000F201A3A0B4A008C02EA13FA13A83298321
:103540008D81882309F48BCFD2019E96BC92AE92D6
:103550009D97D0967C926E929F97EEA1FFA180815D
:10356000882319F081E001C080E0A796E2E10C9485
:10357000E44FA3E0B0E0EFEBFAE10C94C84F1C017C
:103580009B01009709F4CFC04115510509F4CBC048
:10359000FA0101900020E9F7E41BF50BCF010B962F
:1035A0006DE070E00E947F4F862F8F5F8B83D90183
:1035B00093964D905C9094974114510451F0AA2435
:1035C000BB246501EE24FF24870166247724430190
:1035D0000BC0F101E688F788008D118D6288738831
:1035E00084889588570168011A82E614F704080553
:1035F000190509F06BC04114510409F494C0E11499
:10360000F1040105110571F1C101B20158DB009708
:1036100041F5C101B20141E050E0EBDB8C010097C4
:1036200009F481C002501040B80180E090E00E5FC4
:103630001F4FD10150962D913C91519740E050E0A1
:103640000E94604F5B016C01F10182899389A4891A
:10365000B589A80EB91ECA1EDB1EC101B80183DEE2
:1036600065C02C01F2E04F16510420F4EE24FF2433
:1036700087011DC02EEF3FEF420E531EB20180E0C6
:1036800090E0A2E0B0E04A0E5B1EF1012089318992
:1036900040E050E00E94604F7B018C01F101828983
:1036A0009389A489B589E80EF91E0A1F1B1FD10151
:1036B00050968D919C9151973C01882499246E0CD1
:1036C0007F1C801E911E570168011A82D101ED9165
:1036D000FC910190F081E02DC801B701AE014F5F70
:1036E0005F4F21E030E009958823E9F08981853E2C
:1036F00011F0882379F4BA81BF5FBA83EB81BE17DA
:10370000A8F480E290E0A0E0B0E0E80EF91E0A1F05
:103710001B1F6BCF80E290E0A0E0B0E0E80EF91E46
:103720000A1F1B1F5FCFAA24BB246501B501C60178
:103730002396E2E10C94E44FA0E2B0E0E2EAFBE180
:103740000C94C84FDC018B01009719F061157105CD
:10375000F9F400D000D000D02DB73EB72F5F3F4F17
:1037600083EE92E0EDB7FEB792838183F901B383D4
:10377000A283158304830E94484980E02DB73EB799
:103780002A5F3F4F0FB6F8943EBF0FBE2DBF20C13A
:10379000ED91FC9124803580DB019796AD90BD9032
:1037A000CD90DC909A97E62E912EFB01019000209F
:1037B000E9F73197FE2EF61A8F2D90E00C966DE00A
:1037C00070E00E94934F762ECE01019660E270E089
:1037D0004BE050E00E945E48C8016EE270E00E943B
:1037E0009648FC010097E1F09C012F5F3F4F8181DB
:1037F0008823B1F0D9010D900020E9F71197A21BA1
:10380000B30B8A2F8095F80EBE01675F7F4F4A2F5A
:10381000A43008F043E0CB01B90150E00E945548C4
:10382000CE010196B8E0BF1588F06E2D792D4F2D91
:1038300050E00E945548F80180818E3231F5818137
:103840008E3209F482818823F9F01FC0DC018E2DAD
:10385000992D9C01F90188E001900D928150E1F7CA
:10386000D80191968C91982F92959F70803A10F480
:10387000905D01C09F598F708A3010F4805D01C047
:103880008F599F83888701C077248981853E11F4F1
:1038900085E089832CE0822E912C8C0E9D1E85E183
:1038A000F40111928A95E9F7D80190968C9190973E
:1038B0008C8791968D919C9192979C8F8B8F9396EC
:1038C0008D919D910D90BC91A02D8D8F9E8FAF8F6E
:1038D000B8A3672D70E095E0660F771F9A95E1F722
:1038E00080E090E06A0D7B1D8C1D9D1DAE014F5F39
:1038F0005F4F20E230E0F1010995882309F468C0A8
:10390000E980FE01329694018E2D8695E794EE248F
:10391000E794E82A8191E80EE217F307A9F7F72C5C
:103920004E010894811C911C8DE0482E512CBFE063
:103930006B2E4AC0C4016FEF70E040E250E00E947D
:103940005E488F2D90E00197849DD001859DB00D3C
:10395000949DB00D1124A00FB11F91E0F401E90F67
:10396000F11D8C918083892F8F5FF401E80FF11D89
:1039700010829E5F9B3019F09A3121F402C09EE0C4
:1039800001C09CE18C91882321F09F3110F41196A5
:10399000E5CFF982F71419F48F2D806489836C8642
:1039A000EE861D861B8E1C8EC601B501A40120E289
:1039B00030E0F101099580E290E0A0E0B0E0A80ECF
:1039C000B91ECA1EDB1EFA94FF2009F0B3CF81E0B6
:1039D000A096E2E10C94E44FA0E0B0E0E2EFFCE15D
:1039E0000C94CD4F6C015B01EA01009709F495C07E
:1039F0006115710509F491C0FB018081882309F4E8
:103A00008CC04115510581F488C0C501682D772D02
:103A10000E947048009751F4F60183A194A196A7E3
:103A200085A710AA17A679C0842E7D2EC601BE01D7
:103A3000DFDC882351F7F601E080F180C70160E008
:103A400070E041E050E0D5D98C01009709F465C0E1
:103A5000C701B80188DC8BE2FE0111928A95E9F773
:103A600080E188A302501040B80180E090E00E5F32
:103A70001F4FF7012089318940E050E00E94604FDC
:103A8000F7012289338944895589260F371F481F3A
:103A9000591F2FA338A749A75AA73EE2932E988211
:103AA0001AA309A3C701BE0147DE882399F18FA19C
:103AB00098A5A9A5BAA58096A11DB11D8FA398A709
:103AC000A9A7BAA79982F60183A194A19AA389A371
:103AD000C701BE0131DE8823E9F0882D972DB5019D
:103AE0004FE150E00E9487481AA309A3C701B6011D
:103AF000AE013FDD6FA378A789A79AA7611571056D
:103B00008105910539F0C701BE0116DE882311F049
:103B100081E004C0C701B80112D980E0CDB7DEB79B
:103B2000EDE00C94E94FA0E0B0E0E9E9FDE10C9490
:103B3000D04F8C017B01EA01009751F061157105AE
:103B400039F0FB018081882319F04115510521F4DA
:103B500000D087E194E018C0B42EAD2EC801BE019C
:103B600047DC8823D9F0C7016B2D7A2D0E9470485D
:103B70000097A1F7F80183A194A196A785A710AAA1
:103B800017A600D08AEE93E0EDB7FEB7928381834B
:103B90000E94484980E00F900F903AC0F801C08021
:103BA000D1808BE2FE0111928A95E9F78B2D9A2D37
:103BB000B7014FE150E00E948748C601B801AE014D
:103BC000D8DC6FA378A789A79AA76115710581052D
:103BD000910521F400D084EA93E0D6CFC601BE015E
:103BE000ABDD882321F400D088E693E0CDCF00D070
:103BF00000D08AE293E0EDB7FEB792838183F4822E
:103C0000E3820E94484981E00F900F900F900F903F
:103C1000CDB7DEB7EAE00C94EC4FA6E0B0E0E3E10C
:103C2000FEE10C94C84F1C014A015B01009709F4A6
:103C3000CDC0DC0193960D911C919497ED91FC9170
:103C4000208931890115110589F0240135016901A7
:103C5000EE24FF2422273327A9012C193D094E0900
:103C60005F092B833C834D835E8317C0411551054B
:103C70006105710509F493C0E8CFD1018D919C9144
:103C8000B8011DD8009779F02B813C814D815E8170
:103C9000420E531E641E751E8C01C414D504E60426
:103CA000F70458F398C0C301B2016C0D7D1D8E1D41
:103CB0009F1D6150704080409040A70196010E9476
:103CC000A64FD1018D919C91B801A90192D800977E
:103CD00009F47CC00115110521F4F10194A383A31B
:103CE0008C01D10195968D929D92AD92BC92989740
:103CF00081149104A104B10421F494961C921E92A3
:103D00009397F10181919191BF0116DD882309F408
:103D10005DC081149104A104B10429F4F1018081F2
:103D20009181B8013AC0C414D504E604F704B8F18F
:103D3000D101ED90FC90E114F10489F102301105FC
:103D400070F1C701B8010E945F166C018FEF9FEF01
:103D50009A838983D701ED91FC911197000F111F70
:103D6000B80180E090E016962D913D914D915C91C7
:103D70001997620F731F841F951F0480F581E02D32
:103D8000AE014F5F5F4F22E030E00995882339F0A4
:103D9000C114D10421F0C701B6010E949F16F101A0
:103DA00085A596A5A7A5B0A988169906AA06BB065B
:103DB00058F4D1019D968D929D92AD92BC92D09770
:103DC000D2961C921E92D19781E001C080E0269687
:103DD000E2E10C94E44F0115110509F464CF81CFA1
:103DE000A0E0B0E0E6EFFEE10C94D24FEC016B01F5
:103DF000009709F444C06115710509F440C08DA510
:103E00009EA5AFA5B8A9413059F0413018F0423015
:103E1000B1F50CC0FB01E080F1800281138113C079
:103E2000FB01E080F1800281138109C0FB01E08089
:103E3000F180028113818DA19EA1AFA1B8A5E80EEA
:103E4000F91E0A1F1B1F8DA19EA1AFA1B8A58E153B
:103E50009F05A007B10730F4CE01B801A701DDDE50
:103E6000882369F0EDA6FEA60FA718AB1AAA19AA17
:103E7000F601E082F1820283138381E001C080E0D9
:103E8000CDB7DEB7E8E00C94EE4FA6E0B0E0EBE48F
:103E9000FFE10C94C84F9E838D837A8369835C8392
:103EA0004B83009709F442C1672B09F43FC1452BAE
:103EB00009F43CC1DC019D968D909D90AD90BC9025
:103EC000D097FC0185A196A1A7A1B0A58815990559
:103ED000AA05BB0508F42AC10190F081E02D2088D5
:103EE0003188AD81BE81D1960D911C91D29701157B
:103EF000110509F055C093960D911C9194970115E9
:103F00001105A9F481149104A104B10409F00EC1B2
:103F1000CF0160E070E041E050E00E94F9168C01B2
:103F2000ED81FE8194A383A3009709F4FFC0AD81C6
:103F3000BE819D96CD90DD90ED90FC90D097C11400
:103F4000D104E104F10421F52BC0C418D508E6081A
:103F5000F708ED81FE8180819181B8010E945F1692
:103F6000009711F08C0117C0C114D104E104F104D1
:103F700009F0DCC0AD81BE818D919C91B80141E01A
:103F800050E00E94F916009709F4D0C08C0103C0DC
:103F9000210166247724C414D504E604F704A8F6A6
:103FA000089421083108822093200894211C311C98
:103FB000AB80BC80ED81FE81C080D180C114D10472
:103FC000F9F002301105E0F002501040B80180E035
:103FD00090E00E5F1F4FD60150962D913C91519766
:103FE00040E050E00E94604F9B01AC01F6018289E5
:103FF0009389A489B589280F391F4A1F5B1F04C004
:1040000020E030E040E050E07101E818F908AE141B
:10401000BF0408F47501D601ED91FC91C401A0E044
:10402000B0E0280F391F4A1F5B1F0480F581E02D87
:10403000CA01B90149815A8197010995882309F478
:1040400048C0AE18BF08C701A0E0B0E0ED81FE8116
:1040500025A536A547A550A9280F391F4A1F5B1F64
:1040600025A736A747A750ABC701880D991D821514
:10407000930508F180819181B8010E945F16009735
:1040800011F08C0116C0A114B10459F0ED81FE812C
:1040900080819181B80141E050E00E94F9160097BB
:1040A00039F4AD81BE81D2961C921E92D19711C077
:1040B0008C0188249924ED81FE8112AB01ABA114FF
:1040C000B10439F089819A818E0D9F1D9A8389836D
:1040D00071CFED81FE8185A596A5A7A5B0A9E5A024
:1040E000F6A007A110A5E816F9060A071B07C8F4F1
:1040F00085A396A3A7A3B0A7ED81FE81819191919D
:10410000BF011ADB882369F4AD81BE819D96AD9015
:10411000BC909E97AE18BF08FD01E5A6F6A607A7BE
:1041200010AB4B815C814A195B0902C04FEF5FEF16
:10413000CA012696E2E10C94E44F009711F00C942A
:1041400082460895009711F00C94824608950097D6
:1041500011F00C94824608950F931F93CF93DF9331
:104160008C01EB01009721F16115710509F188A11E
:1041700084FF1EC081E390E00E94D545FC019C01B4
:104180000097C1F0AC014E5F5F4FBE018BE2DB01D7
:104190000D90BD01DA010D92AD018150C1F711837F
:1041A000008389A19AA196A785A710AA17A602C085
:1041B00020E030E0C901DF91CF911F910F91089568
:1041C000EF92FF920F931F93CF93DF937C018B01AC
:1041D0000097B9F161157105A1F1DB0190968C9101
:1041E00084FD2FC083E390E00E94D545FC01EC01E3
:1041F000009761F400D08BE494E0EDB7FEB79283B2
:1042000081830E9448490F900F901DC09C012E5F32
:104210003F4FA8018BE2DA010D90AD01D9010D925B
:104220009D018150C1F7F182E08215A616A617A65E
:1042300010AAD80191968D919C91929792AB81ABE7
:1042400002C0C0E0D0E0CE01CDB7DEB7E6E00C940E
:10425000F04FACE2B0E0EFE2F1E20C94C84F1C0189
:10426000009709F45DC1DC0114968D919C9115971E
:10427000892B09F455C116968D919C911797892B1E
:1042800009F44EC18AE190E00E94D5456C019CA7DB
:104290008BA7009709F446C18AE1F60111928A952D
:1042A000E9F7D6012D923C92D10119962D913D91BD
:1042B0004D915C911C9789E0220F331F441F551FBD
:1042C0008A95D1F72AA33BA34CA35DA3CA01B901E8
:1042D000655F7F4F8F4F9F4FED91FC91AE014F5F18
:1042E0005F4F29E130E00995882309F416C1E9817F
:1042F000FA81FFA3EEA32C813D81FB81F8A74E81BB
:104300008F8198859AA789A7E985FA856C857D852F
:104310004E885F88688C798C411451046104710463
:1043200031F4309709F4F9C02F0166247724611520
:10433000710509F4F2C0C901A0E0B0E08E8F9F8F33
:10434000A8A3B9A380E090E0242F30E040E050E043
:104350000E94604F6A8F7B8F8C8F9D8F83017201CB
:104360002E8D3F8D48A159A1E21AF30A040B150BBB
:10437000E61AF70A080B190B8EA19FA1019729A530
:104380003AA5B5E0220F331FBA95E1F7820F931FCC
:104390006EA17FA10E947F4F80E090E0E61AF70AAD
:1043A000080B190B88A5282F30E040E050E0C80129
:1043B000B7010E94A64F79018A0195EFE9169FE0A7
:1043C000F90690E0090790E0190708F4A6C0A5EFE8
:1043D000EA16AFEFFA06A0E00A07A0E01A0720F4F9
:1043E00086E0F101808704C08BE0D10118968C93A0
:1043F000C6010296FC0188E1DF011D928A95E9F76A
:10440000EEA1FFA14F01AA24BB24C301B201A50163
:1044100094010E94604FD60112966D937D938D9307
:104420009C931597C501B4012E8D3F8D48A159A1CC
:104430000E94604F2AA13BA14CA15DA1260F371F0E
:10444000481F591FD60116962D933D934D935C93AB
:104450001997F1018085863029F064E070E080E0F2
:1044600090E004C062E070E080E090E022E030E0A4
:1044700040E050E0E20EF31E041F151FA801970153
:104480000E94604FD6011A966D937D938D939C93F5
:104490001D97EEA1FFA11F96FC93EE931E97F8A522
:1044A0008F2F90E09C014EA15FA1249FC001259F0A
:1044B000900D349F900D112451969C938E9350979C
:1044C0006A8D7B8D8C8D9D8DA50194010E94604F1E
:1044D000D60116962D913D914D915C911997620FE1
:1044E000731F841F951FF601668B778B808F918FCA
:1044F000A9A5BAA59D0140E050E0A5E0220F331F19
:10450000441F551FAA95D1F7620F731F841F951F73
:10451000628B738B848B958B05C0C6010E9482468B
:104520001CA61BA68BA59CA5AC96E2E10C94E44FBF
:10453000A0E0B0E0EEE9F2E20C94CC4F4C01EB01CC
:104540007A01009709F468C06115710509F464C027
:104550008881882309F460C04115510509F45CC0C5
:104560008F3209F421968BE2F70111928A95E9F7CF
:1045700080E1F70180A337018881882309F44EC0C8
:10458000C401B701E9DD6C01009709F445C0CE0113
:104590006FE270E00E946548009739F0482F4C1B8D
:1045A0005C010894A11CB11C2CC0FE0101900020EC
:1045B000E9F731974E2F4C1B5E01A40EB11C21C0B0
:1045C000F30101900020E9F73197E619F709E017A8
:1045D000F107C9F4CE01B301A8010E947948009700
:1045E00091F4C601AADD0C0F1D1FF80180818823FC
:1045F000A9F0F70180A184FF0FC0E501CC24DD24E0
:1046000008C0042F10E0C601B7010E94F8198823E2
:10461000B9F6C60192DDB0CF80E001C081E0CDB730
:10462000DEB7EEE00C94E84F0F9329D3813011F000
:1046300081E02EC08EE594E263EF75E24CEF54E228
:104640002FEA35E200E02ED0909345048093440495
:10465000892BE9F48EE594E263EF75E24CEF54E2C6
:104660002FEA35E20FEF1ED0909345048093440467
:10467000892B69F400D08DE894E0EDB7FEB7928302
:1046800081830E94484981E00F900F9001C080E033
:104690000F910895009711F480E008950E948246DA
:1046A00081E008958F929F92AF92BF92CF92DF9256
:1046B000EF92FF920F93DF93CF93CDB7DEB7609762
:1046C0000FB6F894DEBF0FBECDBF7C016B015A015F
:1046D0004901009709F49EC06115710509F49AC05B
:1046E00004300CF097C007FD1DC0602F772767FDD1
:1046F0007095A4E0660F771FAA95E1F762547E4F8C
:10470000882777FD8095982FAE014F5F5F4F20E19E
:1047100030E0F7010995882309F47CC08D81882356
:1047200009F478C081E190E00E94D545FC01BC010C
:10473000009709F471C081E1DF011D928A95E9F7C4
:10474000F182E082D382C282B582A482978286827D
:1047500007FD5DC08D8180872A8530E040E050E014
:10476000542F432F322F22278B8590E0A0E0B0E01A
:10477000DC0199278827282B392B4A2B5B2B89852D
:1047800090E0A0E0B0E0282B392B4A2B5B2B8C85E6
:1047900090E0A0E0B0E0B82FAA2799278827282B1F
:1047A000392B4A2B5B2BFB012187328743875487A8
:1047B0002E8530E040E050E0542F432F322F222747
:1047C0008F8590E0A0E0B0E0DC0199278827282BB6
:1047D000392B4A2B5B2B8D8590E0A0E0B0E0282B95
:1047E000392B4A2B5B2B888990E0A0E0B0E0B82FF2
:1047F000AA2799278827282B392B4A2B5B2BDB01EB
:104800001D962D933D934D935C93509705C08FEF6C
:10481000808702C060E070E0CB0160960FB6F8942C
:10482000DEBF0FBECDBFCF91DF910F91FF90EF9014
:10483000DF90CF90BF90AF909F908F900895DF92C0
:10484000EF92FF920F931F93D82E7A018B018FEF77
:104850000E944F0A8D2D80640E944F0A812F992754
:10486000AA27BB270E944F0AC801AA27BB270E947C
:104870004F0ABB27A12F902F8F2D0E944F0A8E2DFC
:104880000E944F0ADD2021F088E0D81629F402C0EA
:1048900085E903C087E801C08FEF0E944F0A10E04E
:1048A0008FEF0E944F0A8F3F19F41F5F1A30C1F734
:1048B0001F910F91FF90EF90DF900895A0E0B0E07E
:1048C000E4E6F4E20C94C84F3B014C015A01190193
:1048D00089C03FEF432E31E0532E46205720C201BE
:1048E000A0E0B0E074016301C81AD90AEA0AFB0A21
:1048F00000E012E0041915092016310608F48101C0
:104900008091D2039091D303A091D403B091D503A9
:10491000C816D906EA06FB0609F451C007D1882358
:1049200009F465C02B9881E1B701A60188DF8823CF
:1049300019F4C0E2DEE404C02B9A80E058C021974D
:104940008FEF0E944F0A8E3F19F02097C1F702C0E7
:10495000CD2B71F400D08CEC94E0EDB7FEB79283D0
:1049600081830E9448492B9A80E00F900F903FC0AE
:10497000C2EDD1E08FEF0E944F0A8993F3E0C23D70
:10498000DF07C1F7C092D203D092D303E092D403E1
:10499000F092D50392012E523E4FC501B901A801F4
:1049A0000E945548A00EB11E8FEF0E944F0A8FEF54
:1049B0000E944F0A2B9A8FEF0E944F0A0AC0920161
:1049C0002E523E4FC501B901A8010E945548A00EC4
:1049D000B11E201A310AC801A0E0B0E0680E791EAD
:1049E0008A1E9B1E2114310409F073CF81E0CDB7DC
:1049F000DEB7E2E10C94E44FA0E0B0E0E2E0F5E2E3
:104A00000C94C84F4B015C012A013901212C42E072
:104A1000342E7FC0E401D170CE01A0E0B0E085016A
:104A20007401E81AF90A0A0B1B0B6101CC1ADD0AA2
:104A30006C147D0408F463018091D2039091D30338
:104A4000A091D403B091D503E816F9060A071B0715
:104A5000E9F06CD0882309F461C0209729F480E044
:104A6000C81682E0D80650F4C801B70142ED51E003
:104A700020E032E023DF882309F450C0E092D20323
:104A8000F092D3030093D4031093D50382ED48161C
:104A900081E0580669F09E012E523E4FC901B201D5
:104AA000A6010E9455481092D6036C147D04C1F1F2
:104AB0002B9888E1B801A701C2DE882311F02B9A58
:104AC0002DC08EEF0E944F0AC2EDD1E089910E9465
:104AD0004F0A83E0C23DD807C9F78FEF0E944F0A03
:104AE0008FEF0E944F0A8FEF0E944F0A8F3FD9F736
:104AF0000E944F0A2B9A4C0C5D1CC601A0E0B0E04E
:104B0000880E991EAA1EBB1E6C187D0881E080933A
:104B1000D6036114710409F07DCF02C080E001C0AA
:104B200081E0CDB7DEB7E2E10C94E44F8091D6038B
:104B3000882311F081E008956091D2037091D3032E
:104B40008091D4039091D50342ED51E020E032E012
:104B500053DF882319F081E08093D6030895A0E005
:104B6000B0E0E5EBF5E20C94CA4F5B016C014A0141
:104B7000E901380127014115510569F101151105B8
:104B800051F1FF242115310509F5FF24F3941EC0CE
:104B9000C401B601A5019201F30109958C010097AA
:104BA000E1F0FF2019F4C817D907A8F0C601B50134
:104BB000A401980121DF882371F0C801A0E0B0E0D2
:104BC000A80EB91ECA1EDB1EC01BD10BFF2001F7A9
:104BD0002097F1F602C080E001C081E0CDB7DEB7DA
:104BE000E0E10C94E64FA4E0B0E0E9EFF5E20C94CC
:104BF000C84F4B015C013A013C832B832701DA82C9
:104C0000C98241155105A1F12115310589F102171C
:104C1000130770F1E114F10459F119013094219452
:104C200031083394021B130B6901EE24FF24C501E4
:104C3000B401A3012B813C8141DE8823C9F0C3016B
:104C4000B501A40129813A81F2010995882391F0E7
:104C5000020D131D8B819C81800F911F2B813C8144
:104C60008217930738F08C0C9D1CAE1CBF1CDFCF45
:104C700080E001C081E02496E2E10C94E44F1F93B0
:104C8000239A2B9A83E58CBD8DB58E7F8DBD1092B6
:104C9000D7032B9810E080E040E050E060E070E047
:104CA000CEDD813039F0153019F42B9A80E07CC0CC
:104CB0001F5FF1CF87E340E050E060E070E0BFDDD0
:104CC00089E240E050E060E070E0B9DD82FD09C0BB
:104CD0008091D70381608093D70300D08EE795E061
:104CE00003C000D080E695E0EDB7FEB792838183E4
:104CF0000E9448490F900F901FEF8091D70390E0DA
:104D000083709070892B41F087E340E050E060E0D1
:104D100070E095DD89E201C081E040E050E060E0B4
:104D200070E08DDD80FF09C0112329F42B9A00D09B
:104D300087E295E00EC01150E0CF80E140E052E004
:104D400060E070E07CDD882371F02B9A00D081EF69
:104D500094E0EDB7FEB7928381830E94484980E0DA
:104D60000F900F9021C02B9A8CB58C7F8CBD8DB588
:104D700081608DBD8FEF9FEFAFEFBFEF8093D203C8
:104D80009093D303A093D403B093D50381E0809391
:104D9000D60360E070E080E090E042ED51E020E07A
:104DA00032E08CDD811181E01F910895DC011196C4
:104DB000ED91FC91129765A176A187A190A5089528
:104DC00080913B0490913C04009729F0B6D9109251
:104DD0003C0410923B048091D8039091D903009732
:104DE00029F0B5D91092D9031092D80380914404C8
:104DF00090914504009729F04DDC109245041092E3
:104E000044040895A5E0B0E0E8E0F7E20C94D54F43
:104E100080913B0490913C04892B11F401E03CC04B
:104E200000D08CEB95E0ADB7BEB712969C938E93F5
:104E300011970E9448490F900F9060E070E080E069
:104E400090E08E010F5F1F4FA80125E030E036DDB6
:104E5000F82E60E072E080E090E0A80125E030E00C
:104E60002DDD882319F000E0FF2009F401E000D0D7
:104E700000D0EDB7FEB731968DE995E0ADB7BEB77E
:104E800012969C938E931197028313820E94484935
:104E90000F900F900F900F90802F2596E5E00C94C7
:104EA000F14FABE2B0E0E7E5F7E20C94C84F7C01CC
:104EB0002DB63EB6FE0131968BE2DF011D928A953A
:104EC000E9F780E189A34F0103C00894E11CF11CBC
:104ED000F70180818F32C9F38091D8039091D90373
:104EE000B4013AD95C01009779F400D08CE296E0E5
:104EF000ADB7BEB712969C938E9311970E94484906
:104F000041E00F900F9099C0C7016FE270E00E94DE
:104F10006548009719F0482F4E192EC0F7010190EF
:104F20000020E9F731974E2F4E1926C0C401B70172
:104F3000A6010E947948009709F5C501FED889A10C
:104F400084FD12C000D000D088E096E0EDB7FEB737
:104F500092838183F482E3820E94484941E00F906A
:104F60000F900F900F9069C0EC0CFD1CD7018C9135
:104F7000882309F0ADCF60C0C42EDD24C501B40183
:104F80000E94F819882391F67DB66EB65DB64EB6CE
:104F9000C6010196EDB7FEB7E81BF90B0FB6F89402
:104FA000FEBF0FBEEDBF0DB71EB70F5F1F4FC8018D
:104FB000B7014C2D50E00E945548F801EC0DFD1D45
:104FC0001082C501B801A4010E94EC1C8823C9F419
:104FD000C501B3D800D000D0EDB7FEB7319682EE50
:104FE00095E0ADB7BEB712969C938E93119702834E
:104FF00013830E94484941E00F900F900F900F904B
:1050000009C0C5019AD8EC0CFD1CF70180818823EA
:1050100051F440E0852D942D9C010FB6F8943EBFCD
:105020000FBE2DBF0AC0872D962D9C010FB6F89498
:105030003EBF0FBE2DBF4CCF40E0842F0FB6F8947B
:105040003EBE0FBE2DBEAB96E2E10C94E44FFC01D8
:10505000818192810E940D1E90E0882309F491E0E5
:10506000892F0895A4E0B0E0E8E3F8E20C94D84F6B
:1050700049835A836B837C83FC0181819281BE01C9
:105080006F5F7F4F422F0E94F01E882311F080E057
:1050900001C08FEF2496E2E00C94F44FFC01818173
:1050A0009281A9010E94451F9C01442737FD40952C
:1050B000542FB901CA010895FC0181819281A9018F
:1050C0000E949D179C01442737FD4095542FB9013C
:1050D000CA0108950F931F938C01FC018181928175
:1050E00031D8C8010E9482461F910F910895ABE20A
:1050F000B0E0EDE7F8E20C94D64FBC018091D80304
:105100009091D9038E010F5F1F4FA80111DA8823F8
:1051100019F420E030E007C08091D8039091D903C2
:10512000B8011AD89C01C901AB96E4E00C94F24F87
:10513000ABE2B0E0EEE9F8E20C94D14F7C01B62E80
:1051400003C00894E11CF11CD7018C918F32C9F384
:10515000C0903B04D0903C04C7016FE270E00E9415
:1051600096488C01009791F0FC011082C701BFDFC7
:105170006C018FE2D8018C93C114D10419F400E0C2
:1051800010E05CC078010894E11CF11CBB2039F0F0
:10519000C601B701AE014F5F5F4F0E94931DC6016C
:1051A0000E94BC188E010F5F1F4F1DC0C801B701C0
:1051B0000E9470480097B9F489A184FD1AC08091BB
:1051C000D8039091D903B8010E94E0207C0189E0C6
:1051D00090E00E94D545FC018C01009761F010829F
:1051E000F282E18208C0C601B8010E94F819882342
:1051F000E9F600E010E0BB20B9F001151105A1F0BF
:10520000D8011196ED91FC91129785A196A1A7A1C5
:10521000B0A50097A105B10539F0CF0140E050E0FD
:1052200060E070E00E940D1E80913B0490913C0470
:10523000C816D90619F0C6010E949D20C801AB9678
:10524000E9E00C94ED4F60E073CF61E071CF8091A5
:105250004404909145040E9429219093D90380939E
:10526000D803892B49F083E091E041DF90933C041F
:1052700080933B04892B69F400D08CE896E0EDB76D
:10528000FEB7928381830E94484981E00F900F907E
:10529000089500D083E596E0EDB7FEB79283818351
:1052A0000E94484980E00F900F900895FC015381BF
:1052B000560F5093DF03272F33274281420F40932D
:1052C000DE03A181A093DD03E081E093DC03842F62
:1052D00090E08217930748F48A2F8F5F8093DD0355
:1052E000882319F4EF5FE093DC03852F90E0707062
:1052F0008617970790F4842F8F5F8093DE038823AF
:1053000061F48091DD038F5F8093DD03882329F4AE
:105310008091DC038F5F8093DC0308959C014150F2
:105320005040460F571FFB010EC0708160E0818125
:10533000DB01A80FB11D2A0F3B1F2A173B0710F4F2
:105340002F5F3F4F3296E417F50778F3E417F50720
:1053500049F4908180E0280F391F2817390710F48D
:105360002F5F3F4FC901089580E090E067E376E04A
:1053700044E150E0D3DF009719F42FEF3FEF02C074
:10538000382F292FC90108950F931F9300913A06D2
:1053900010E0045110403091390620E0020F131F35
:1053A0009801280F311DC90163E476E048E050E020
:1053B000B5DF6BE476E0A801B1DF009719F42FEFB9
:1053C0003FEF02C0382F292FC9011F910F91089577
:1053D000E5EFF5E011821082349686E0ED31F807B2
:1053E000C9F710927A04109201051092880580E0A6
:1053F00094E0909356048093550408959C01E5EF42
:10540000F5E0A0E0B0E080819181892B71F4AA0FD2
:10541000BB1FAA0FBB1FFD01EB50FA4F3183208346
:10542000A950BA4F6D937C93089511963496AA3083
:10543000B10549F70895BC0180915D0490915E0427
:10544000089634DFE0915D04F0915E048091DC0306
:105450008087E0915D04F0915E048091DD03818797
:10546000E0915D04F0915E048091DE038287E0911B
:105470005D04F0915E048091DF03838708950F93AC
:105480001F93CF93DF932FE536E030935C04209396
:105490005B043093530420935204C0915D04D09177
:1054A0005E048330A1F48B8D8F70833009F01DC6AC
:1054B00088899989892B09F018C688E0809354045B
:1054C000CB57DF4FE881F981C558D0409EC4823068
:1054D00009F0A0C080915A048F5F80935A048823FA
:1054E00099F4809159048F5F80935904882361F463
:1054F000809158048F5F80935804882329F4809109
:1055000057048F5F8093570410924704109246040B
:105510001092200810921F082B8D273011F0253093
:1055200041F48C8D8F5F8C8F883709F0DEC51B8E20
:10553000DCC5222309F4D9C588899989892B09F406
:1055400061C08C8D81508C8F8F5F09F0CEC53D8DF1
:10555000383029F021502230A0F4353091F41B8EE0
:1055600080E880935404E0915D04F0915E04EB5771
:10557000FF4F0190F081E02D309709F453C4099555
:1055800051C4353010F080E307C083E090E002C0E2
:10559000880F991F3A95E2F78C8F8D8D8F5F8D8FD5
:1055A0008B8D90E08F70907083309105D1F08430B6
:1055B000910544F48130910509F42AC2029709F05B
:1055C00094C50CC08630910509F4C1C3883091059B
:1055D00009F4BDC3049709F088C5B9C310925806F1
:1055E0001AC284E080935404E0915D04F0915E045B
:1055F000EB57FF4F0190F081E02D309709F447C43D
:10560000099545C42F70233009F06FC588E0809359
:105610005404F2C389010852104080913706853442
:1056200009F063C59091390680E020913A06AC01FB
:10563000420F511D809146049091470484179507AD
:1056400008F453C5509347044093460480913D06A7
:1056500090E08F739070892B09F047C580913E06CA
:10566000882309F042C52091470630914806809171
:105670002506909126062817390709F036C520918E
:10568000490630914A0680912706909128062817EE
:10569000390709F02AC568DE8F5F9F4F09F025C5DD
:1056A000809140068630D1F1813009F01EC580918D
:1056B0004B06883009F019C510924B0680914D06B3
:1056C00090914E06EFEF873F9E0710F0099601C0BC
:1056D000089690934E0680934D06809143069091D4
:1056E0004406909348068093470680914506909122
:1056F000460690934A06809349068091250690912C
:105700002606909344068093430680912706909145
:1057100028069093460680934506EBC486E034DE67
:105720008F5F9F4F09F0E1C4CFE5D4E08B8D8823D4
:1057300029F120914D0630914E068C819D812817CC
:105740003907E1F420914B0630914C068E819F8100
:105750002817390799F4209143063091440688812F
:1057600099812817390751F4209145063091460652
:105770008A819B812817390709F466C1C957DF4F11
:1057800025E0CD36D20791F288F2809158068F73CA
:10579000823091F440914D0650914E06A5EFB5E050
:1057A000FD01808191814817590709F469C0349639
:1057B00086E0ED31F807A9F78091580682FD95C47F
:1057C00084E1F80181A388E290E0909347048093FC
:1057D000460480E580A39091520680915606838FFF
:1057E0004091510680915506828F468F3091500628
:1057F00080915406818F358F20914F0680915306FA
:10580000808F248F9F5F978F992361F4842F8F5F00
:10581000868F882339F4832F8F5F858F882311F437
:105820002F5F248F20914B0630914C0680914D06BE
:1058300090914E06F801958B848B378B268B809147
:1058400043069091440690934806809347068091C2
:1058500045069091460690934A06809349068091AA
:1058600025069091260690934406809343068091E6
:105870002706909128069093460680934506F8C324
:10588000EFE5F4E0C0E0D0E020E0838D882339F438
:1058900087E8289FE0011124C15ADB4F0EC08730F2
:1058A00039F4209721F0948D8C8D891708F4EF013D
:1058B0002F5FE957FF4F233041F7209709F415C4B4
:1058C000D0935E04C0935D04E0E0F0E08D919C9184
:1058D00011974817590779F4CB57DF4FEE0FFF1F89
:1058E000EE0FFF1FE950FA4F8081918199838883E1
:1058F000C558D04005C031961496EA30F10531F70D
:1059000083E08C8F8A8F188E84E0898F1D8E1B8A8E
:105910001A8A80914D0690914E069D838C838091CA
:105920004B0690914C069F838E8380914306909105
:1059300044069983888380914506909146069B830F
:105940008A8381E08B8F809157048C8780915804E3
:105950008D87809159048E8780915A048F8781E0CA
:1059600090E0998B888B809152068B8780915106AD
:105970008A8780915006898780914F06888781E0C9
:1059800090E059DD20915706822F90E0807F907043
:1059900081359105ECF122952F7030E02550304093
:1059A000220F331F220F331F90E02DC0DF01A75DB0
:1059B000B94FD6968C91D697882351F1813011F446
:1059C0009F5F21C08230C9F4D7968C91D7978430DD
:1059D000A1F4D8969C91D89780E0D9962C9130E08C
:1059E000282B392BF1E02F3B3F0710F02EEB31E055
:1059F0003D8B2C8B3F8B2E8B0BC0E75DF94F87A91E
:105A0000882331F0980FE92FF0E0E217F30774F2E2
:105A100080E18093580680915806826080935806F2
:105A200082E080935F0684E08093600681E080934B
:105A300061068EEB809362068CE290E090934704BF
:105A40008093460480E6B9C2D0935E04C0935D049F
:105A50001092540480915806482F50E082FF03C0F2
:105A60001B8E80E241C220914604309147042451AC
:105A700030408091570682958F70880F880F281BC1
:105A8000310930934704209346048B8D8F70823008
:105A900029F44F7350704231510509F1232B39F429
:105AA0008091580690E083709070892BC1F090919E
:105AB0004F068885981709F076C29091500689851F
:105AC000981709F070C2909151068A85981709F0CD
:105AD0006AC2909152068B85981709F064C2809132
:105AE000580684FF50C0688979896115710509F4E9
:105AF0004AC0CE010C96DADB209153068091DC037C
:105B0000281709F040C0909154068091DD03981742
:105B1000D1F5909155068091DE039817A1F59091EB
:105B200056068091DF03981771F52C878091DD036D
:105B30008D878091DE038E878091DF038F878D8D27
:105B40008823D1F4288D9A8D8C8D981B822F869571
:105B500086958695981B392F320F388F898D282F7F
:105B600026952695821B97FD9195890F898F3695ED
:105B700036953695830F8A8F81E0809354048A8D01
:105B80008C8F198A188A8B8D282F30E0C901AA279B
:105B900097FDA095BA2F8F709070A070B070FC0127
:105BA0003197E830F10508F0A0C2E85CFF4F0C9493
:105BB000FF4F8091540480FF98C283E08B8F80E474
:105BC00080935404198A188A20914604309147041E
:105BD0002115310509F40CC1809154048260809331
:105BE0005404C90128DC04C18091540480FF67C0BB
:105BF000809158068F73823109F061C02091570659
:105C0000822F90E0807F907081359105ECF1229594
:105C10002F7030E025503040220F331F220F331FEA
:105C200090E02DC0DF01A75DB94FD6968C91D69735
:105C3000882351F1813011F49F5F21C08230C9F473
:105C4000D7968C91D7978430A1F4D8969C91D89709
:105C500080E0D9962C9130E0282B392B41E02F3B66
:105C6000340710F02EEB31E03D8B2C8B3F8B2E8BCD
:105C70000BC0E75DF94F87A9882331F0980FE92F12
:105C8000F0E0E217F30774F283E08B8F80914F0608
:105C90008887809150068987809151068A878091F4
:105CA00052068B8781E090E0C6DB82E48093540447
:105CB000198A188A109247041092460499C080E20B
:105CC00080935404E0915D04F0915E04EB57FF4F24
:105CD0000190F081E02D309709F00995E0915D0485
:105CE000F0915E04138E68CD8091580680FF33C01A
:105CF00024FD31C088899989892B09F0F6C18091EA
:105D0000460490914704019696DB20915404822F1B
:105D10008061809354048091460490914704892BBC
:105D200019F0226120935404E0915D04F0915E0427
:105D3000EB57FF4F0190F081E02D309709F0099566
:105D400081E090E0998B888B88E08B8F1D8E81E1BC
:105D5000809358062BC185FF21C060915D06362FC8
:105D600020E040915E0650E0242B352B80915B04AF
:105D700090915C04820F931F90935C0480935B046A
:105D8000962F80E0842B952B209146043091470478
:105D9000281B390B30934704209346042091460476
:105DA000309147042115310551F08B8D84FD07C0DA
:105DB00080915404826080935404C9013CDB90912B
:105DC000590680E020915A06820F911D2E893F8945
:105DD0002817390710F0009709F4C9019D8B8C8BA7
:105DE0008091540490E083709070892B09F47DC1F8
:105DF0001092200810921F08E0915D04F0915E045B
:105E0000EB57FF4F0190F081E02D309709F0099595
:105E100080915404282F85FF07C01092200810920B
:105E20001F081B8E84E194CF84FF0AC010922008C3
:105E300010921F0881E090E0998B888B84E085CFD9
:105E400080911F0890912008892B01F120FF02C04A
:105E5000198A188A888999890097A1F42C893D8923
:105E600080911F08909120082817390720F430935B
:105E7000200820931F0880911F0890912008998B7B
:105E8000888B04C09093200880931F081D8E8091FA
:105E900052049091530490935C0480935B0480912E
:105EA0001F0890912008892B59F0888999890097BB
:105EB00039F08896909347048093460488E10BC09C
:105EC0008091540481FF11C188E290E090934704CF
:105ED0008093460480E1809358066EC080915404FC
:105EE00080FF03C11B8E80E180935404E0915D0428
:105EF000F0915E04EB57FF4F0190F081E02D309759
:105F000009F4F3C00995F1C08091460490914704CB
:105F1000009709F090DA809158069091540480FF20
:105F20000BC090FF06C087E08B8F1C8E198A188AE1
:105F300018C086E08B8F15C090FF26C085E08B8F40
:105F4000198A188AD2C0809146049091470400971C
:105F500009F071DA8091580680FF16C087E08B8FB8
:105F60001C8E81E090E067DA80E180935404E09138
:105F70005D04F0915E04EB57FF4F0190F081E02D3E
:105F8000309789F009950FC080914604909147049D
:105F9000892B49F4AAC08091540480FFA6C087E0F1
:105FA0008B8F1C8EA2C080E1F80181A388E290E073
:105FB000909347048093460480E580935706888534
:105FC000809353068985809354068A85809355066D
:105FD0008B85809356068C8580934F068D858093A4
:105FE00050068E85809351068F858093520686E0F9
:105FF000809340068C819D8190934C0680934B0644
:106000008E819F8190934E0680934D068091250648
:10601000909126069093440680934306809127062C
:106020009091280690934606809345068881998131
:1060300090934806809347068A819B8190934A06F5
:10604000809349068B8D84FF05C010925A061092EA
:1060500059060EC08A899B89009721F090935906B2
:106060008A8904C081E0809359068EEB80935A069A
:1060700080E480933F0680914704809339068091A5
:10608000460480933A0610925E0610925D061092C6
:106090005C0610925B0686E077D980959095909388
:1060A0005C0680935B0685E4809337061092380681
:1060B00010923E0610923D068091DA039091DB0328
:1060C00001969093DB038093DA0390933B068093D1
:1060D0003C06109242061092410646D98095909552
:1060E000909342068093410604C010924704109298
:1060F000460410925404DF91CF911F910F9108959F
:10610000AC01FB011616170684F460931F08F09388
:10611000200820915204309153048217930729F0EC
:10612000C901BA01AF010C94554808956115710574
:1061300099F12DB73EB72C5030400FB6F8943EBFC2
:106140000FBE2DBFEDB7FEB73196ADB7BEB71296F5
:106150009C938E9311978EEC96E093838283758344
:1061600064836F5F7F4F778366836F5F7F4F718735
:1061700060876F5F7F4F738762870E94E8492DB702
:106180003EB7245F3F4F0FB6F8943EBF0FBE2DBF02
:10619000843011F480E008958FEF0895CF93DF935A
:1061A000DC010097E9F400D000D000D0EDB7FEB7D5
:1061B0003196ADB7BEB712967C936E931197538309
:1061C000428385E091E0958384830E946B49CDB73B
:1061D000DEB726960FB6F894DEBF0FBECDBF32C035
:1061E0002DB73EB72E5030400FB6F8943EBF0FBECD
:1061F0002DBFEDB7FEB73196CDB7DEB77A83698391
:106200005383428382EE96E0958384838C918683C8
:10621000178211968C9111978087118612968C9116
:1062200012978287138613968C91848715860E9415
:1062300099492DB73EB7225F3F4F0FB6F8943EBF46
:106240000FBE2DBFDF91CF910895DC016D917C9140
:106250001197E0EEF3E0AF01808191816817790733
:1062600049F412962D913C911397828193812817BE
:10627000390739F03B9684E0E833F80761F740E0EE
:1062800050E0CA010895A0E0B0E0E9E4F1E30C9425
:10629000D34F8C01E62ED72EA0EEB3E0FD01408156
:1062A000518141155105F9F02281338121153105C4
:1062B000D1F0E8018881998184179507A1F48A813A
:1062C0009B818217930779F4EF0124968E2D9D2DE3
:1062D0009C01D90186E00D9009928150E1F78091EF
:1062E000380482874BC03B9684E0E833F807B9F660
:1062F00020E0ED018D919C911197892B31F412963C
:106300008D919C911397892B19F12F5F1B96283043
:1063100081F7F0903804AF2DB0E0EAEEF3E040E012
:1063200070E060E050819D01251B3109872F90E0CE
:10633000821793071CF47F2D751B642F4F5F3B96CC
:10634000483081F78BE0689FE0011124C052DC4F98
:10635000F80180819181A281B381FE0181939193A3
:10636000A193B1932E2D3D2DC901DC0186E00D9046
:1063700001928150E1F7809138048A87CDB7DEB76A
:10638000E7E00C94EF4F80914306909144062091F2
:1063900025063091260682279327209121063091E9
:1063A000220682239323892BB9F48091450690918C
:1063B00046062091270630912806822793272091B0
:1063C00023063091240682239323892B29F483E426
:1063D00096E06FE276E057CF0895CF93DF938091F8
:1063E0004604909147048A9728F41092470410922B
:1063F00046048EC01092470410924604C9E2D6E0CB
:1064000080913D0690913E0621E08030920729F070
:106410008050924009F07CC05FC020914F063091BF
:10642000500680912506909126062817390709F015
:106430006FC02091510630915206809127069091AD
:1064400028062817390709F063C0CE014C96BE0113
:106450006A5E7F4F18DF80E092E090933E06809363
:106460003D06DE019096FE01769686E001900D9243
:106470008150E1F7AFE3B6E0E8E4F4E086E00190B4
:106480000D928150E1F7AFE2B6E0E8E4F4E086E097
:1064900001900D928150E1F7E9E2F6E0DF0190967C
:1064A00086E00D9001928150E1F7E5E4F6E09285F7
:1064B00080818287919386E0E934F807C1F788E00C
:1064C00096E090933606809335068AE290E09093AA
:1064D0004704809346041CC020914F06309150061B
:1064E00080912506909126062817390789F4209176
:1064F0005106309152068091270690912806281760
:10650000390731F4CE014C96BE016A5E7F4FBBDE87
:10651000DF91CF910895A4E0B0E0E1E9F2E30C94BB
:10652000D84F80914706805E8031B0F481E080933F
:10653000290610922A068EE580932B068091480644
:106540008F7780932C068091490680932D06809149
:106550004A0680932E06DBC0409125065091260600
:10656000E0912106F0912206CF0180959095842B31
:10657000952B20914706309148062817390799F442
:10658000809123069091240680959095209127066E
:1065900030912806822B932B2091490630914A0690
:1065A0002817390791F0609147067091480680914D
:1065B0002A0190912B016817790789F48091490687
:1065C00090914A068F5F9F4F51F4A9E2B6E0EEE248
:1065D000F1E086E001900D928150E1F798C04627E6
:1065E00057274E235F23452B91F440914906509144
:1065F0004A068091270690912806842795272091A6
:1066000023063091240682239323892B69F08091FD
:106610001D0690911E069A83898380911F06909192
:1066200020069C838B8304C07A8369835C834B83BD
:10663000CE0101960ADE009709F060C089E296E07B
:106640006FEF70E046E050E00E945E48E9E4F6E05B
:1066500086E0DF011D928A95E9F77A97A8E4B4E015
:1066600086E00D9001928150E1F7AFE3B6E0E8E4F7
:10667000F4E086E001900D928150E1F789819A81E2
:106680009093500680934F068B819C819093520685
:106690008093510680912506909126069093460698
:1066A000809345068091270690912806909348068E
:1066B0008093470680E091E090933E0680933D06EC
:1066C000909338068093370688E090E090933A06DE
:1066D0008093390686E080933B0684E080933C06F5
:1066E00088E096E090933606809335068AE290E043
:1066F000909347048093460481E022C0A9E2B6E06B
:10670000FC01349686E001900D928150E1F7AFE2F2
:10671000B6E0E8E4F4E086E001900D928150E1F704
:1067200088E090E090933606809335068091460489
:10673000909147040E96909347048093460480E01E
:106740002496E2E00C94F44F809138048F5F80939C
:106750003804A0EEB3E012968D919C9113972D9181
:106760003C911197822B932B892B81F080913804D7
:1067700090E01A962C911A97821B910988379105FF
:106780002CF0FD0110821182128213821B9684E08C
:10679000A833B80701F7089580E090E02BE030E0DF
:1067A000829FF001839FF00D929FF00D1124E05223
:1067B000FC4F10821182128213820196883091055B
:1067C00079F708950E94CD0880E090E00895A0E058
:1067D000B0E0EDEEF3E30C94D04F8C017B01B42ECE
:1067E000A52EDC018C91873121F087E18C931196E5
:1067F0001C92F8018181E82FF0E0EE0FFF1FEE0FF1
:10680000FF1FEE52F14F8F5FD80111968C932591A7
:106810003491D22EC32EC9010E942648AC012B2DE3
:106820003A2DC901EC014817590708F4EA01C701DC
:106830006D2D7C2DAE010E940B48F8018181E82F5F
:10684000F0E0EE0FFF1FEE0FFF1FEE52F14F8591AC
:106850009491892B31F086EF9FEF9C012C1B3D0B0F
:10686000E901CE01CDB7DEB7EAE00C94EC4F2DB7CD
:106870003EB7285030400FB6F8943EBF0FBE2DBF34
:10688000EDB7FEB73196ADB7BEB712967C936E9357
:106890001197538342838EEE96E0958384838AE03A
:1068A00091E0978386830E9499492DB73EB7285F70
:1068B0003F4F0FB6F8943EBF0FBE2DBF08956F92A5
:1068C0007F928F929F92AF92BF92DF92EF92FF9250
:1068D0000F931F93CF93DF937C015B013A01FC017F
:1068E00001900020E9F73197E81BF90B329718F473
:1068F00020E030E054C0DD248D2C9924F401EE0F0B
:10690000FF1FEE0FFF1FEE52F14FC591D49120975C
:10691000C9F0CE010E9426488C01C701BE01A80122
:106920000E94FE47892B61F4E00EF11EF401EE0F88
:10693000FF1FEE0FFF1FEC52F14F2591349104C061
:10694000D394DACF20E030E08BB190E489278BB983
:106950002115310519F42FEF3FEF06C0C701B5012E
:10696000A301F90109959C01A114B104C1F08FEFB5
:106970002F3F380751F4C50161EF76E04BE050E05E
:106980000E940B482BE030E00AC02115310539F494
:106990008FE4F50180838BE4818322E030E0C9013C
:1069A000DF91CF911F910F91FF90EF90DF90BF90FB
:1069B000AF909F908F907F906F9008950F931F934B
:1069C000CF93DF93EC018C010A5D1F4FC8016DEF7F
:1069D00076E04DE050E00E944748892B19F42BE007
:1069E00037E016C1C80169E177E04EE050E00E944F
:1069F0004748892B19F428E237E00AC1CE016EE33B
:106A000077E045E050E00E944748892B19F424E4E0
:106A100037E0FEC0CE016DE477E046E050E00E9432
:106A20004748892B19F424E537E0F2C0CE0161E62E
:106A300077E04EE050E00E942F48892B69F1CE01AB
:106A40006AE777E045E050E00E942F48892B21F16A
:106A5000CE0160E877E046E050E00E942F48892BA5
:106A6000D9F0CE0167E877E045E050E00E942F487A
:106A7000892B91F0CE016DE877E044E050E00E9470
:106A80004748892B49F0CE0162E977E043E050E0C6
:106A90000E942F48892B19F420E737E0B9C0CE01B6
:106AA00066E977E042E050E00E944748892BD9F040
:106AB000CE0161EB77E042E050E00E944748892B2D
:106AC000F1F0CE016DEC77E042E050E00E944748E3
:106AD000892B09F1CE0168EE77E042E050E00E9498
:106AE0004748892B19F429E937E092C0CE016BEEB3
:106AF00077E042E050E00E944748892B19F424EBEC
:106B000037E086C0CE016EEE77E042E050E00E94B2
:106B10004748892B19F420ED37E07AC0CE0161EFA8
:106B200077E044E050E00E944748892B19F426EFB3
:106B300037E06EC0CE0163E078E042E050E00E94B2
:106B40004748892B49F0CE0161E178E042E050E00E
:106B50000E944748892B19F426E038E059C0CE013D
:106B600064E178E046E050E00E944748892B91F0CC
:106B7000CE016BE278E046E050E00E944748892B66
:106B800049F0CE0162E378E043E050E00E944748DC
:106B9000892B19F42BE138E03BC0CE0166E378E0A5
:106BA00043E050E00E944748892B19F42AE338E07B
:106BB0002FC088818F3F31F48981883D19F424E406
:106BC00038E026C0CE016FE478E042E050E00E9459
:106BD0004748892B19F422E538E01AC0CE0161E656
:106BE00078E044E050E00E944748892B19F426E6FB
:106BF00038E00EC0CE0160E778E043E050E00E944C
:106C00004748892B19F020E838E002C024E738E033
:106C1000C901DF91CF911F910F910895EF92FF92DB
:106C20000F931F938091540480FF04C080E18093F0
:106C3000540462C0E0915B04F0915C041082809186
:106C40005B0490915C046DE979E00E9414488091A6
:106C50005B0490915C046DE77AE00E941448E09038
:106C60005B04F0905C04D7010D900020E9F78D01E2
:106C7000015010400E191F0989E09AE00E94264831
:106C800000D000D000D0EDB7FEB73196E00EF11E77
:106C9000ADB7BEB71296FC92EE9211972BE838E092
:106CA00033832283958384830E94C7498DB79EB71F
:106CB00006960FB6F8949EBF0FBE8DBF80915B0401
:106CC00090915C046EE87AE00E94144880915B0425
:106CD00090915C0469E07AE00E94144880915B0422
:106CE00090915C04FC01DF010D900020E9F7119701
:106CF000AE1BBF0BBD0104DA1F910F91FF90EF9007
:106D00000895EF92FF920F931F938091540480FF98
:106D100004C080E18093540462C0E0915B04F09170
:106D20005C04108280915B0490915C0466E17AE0DF
:106D30000E94144880915B0490915C046DE77AE0B6
:106D40000E941448E0905B04F0905C04D7010D9021
:106D50000020E9F78D01015010400E191F098DE642
:106D60009AE00E94264800D000D000D0EDB7FEB7D0
:106D70003196E00EF11EADB7BEB71296FC92EE92C0
:106D800011972FE838E033832283958384830E9410
:106D9000C7498DB79EB706960FB6F8949EBF0FBE33
:106DA0008DBF80915B0490915C046EE87AE00E9454
:106DB000144880915B0490915C046DE67AE00E9437
:106DC000144880915B0490915C04FC01DF010D90FC
:106DD0000020E9F71197AE1BBF0BBD0191D91F91A0
:106DE0000F91FF90EF9008950F93E0915D04F09163
:106DF0005E04878D90A1825C984399F461A172A191
:106E00006115710571F082E020E030E040E050E073
:106E100000E00E946F0AE0915D04F0915E0412A20E
:106E200011A2E0915D04F0915E04878D90A18F51D5
:106E30009B4361F481A192A1009741F00E949D20A3
:106E4000E0915D04F0915E0412A211A20F910895E9
:106E5000A0E0B0E0EEE2F7E30C94D14F809154044F
:106E600085FD02C087FF01C0BFDF8091540484FF0D
:106E700001C0BADF8091540486FF1BC0E0915D041D
:106E8000F0915E0410A2178EE0915D04F0915E0413
:106E9000868D8E7F868FE0915D04F0915E04868DF5
:106EA0008B7F868FE0915D04F0915E04868D8D7FEF
:106EB000868F8091540481FFDBC0C0915D04D09126
:106EC0005E048F8D98A1892B19F08E8D81FFD0C023
:106ED00080914604909147040A97D0F0C0905B04DB
:106EE000D0905C04C60163EA7AE045E050E00E947D
:106EF0002F48892B69F485E0E82EF12CEC0CFD1C61
:106F0000C70160E270E00E946548FC01009729F427
:106F10008EE096E398A38F8FABC010828DE99AE044
:106F20000E942648C82FD0E0C70167E97AE0AE0189
:106F30000E944748892B29F4C7018C0F9D1FE9D275
:106F400097C0C7016FE270E00E949648FC01A091D3
:106F50005D04B0915E04009711F0818102C0F601DA
:106F6000858193968C9300915D0410915E04C70116
:106F70000E940B0BF80192A381A3E0915D04F091B4
:106F80005E0481A192A1892B39F5E70109900020C7
:106F9000E9F72197CE19DF09CE0DDF1DBA902196B2
:106FA000FFE2BF1611F08FE28993CE0160E97AE02B
:106FB0000E941F4800915D0410915E04C7010E9469
:106FC0000B0BF80192A381A3E0915D04F0915E04A4
:106FD00081A192A1892B29F082EC98E390A3878F5D
:106FE00047C0CE15DF0519F4F601158202C02197BE
:106FF000188200915D0410915E04E7012197CE0193
:107000000E947728F80192A381A3A0915D04B0911A
:107010005E04892B39F1CD018396BE014BE450E02B
:107020000E948748E0915D04F0915E04E359FF4FB0
:107030001082A0915D04B0915E04FFE2BF1679F06A
:1070400080ED9AE390969C938E935F97E0915D0418
:10705000F0915E0481A192A10E949D2009C08FE160
:107060009BE302C081E896E390969C938E935F9792
:1070700080915404282F30E082FD09C0C90183703B
:107080009070892B21F428743070232B71F0E091DB
:107090005D04F0915E04278D30A12115310529F0A2
:1070A000868D81FD02C0F9010995CDB7DEB7E9E013
:1070B0000C94ED4F0F931F9308E217E380E090E5E7
:1070C000B8010E94FE298FE190E4B8010E94FE29D8
:1070D0001F910F9108950F931F93E0915D04F0911C
:1070E0005E0461A172A124A135A146A157A180E04F
:1070F00000E00E946F0AE0915D04F0915E0461A1DE
:1071000072A140915B0450915C040489158920E0D0
:1071100030E080E00E94AB0A9B01AC016115710573
:107120008105910529F480E2809354045DDE27C037
:10713000E0915D04F0915E0484899589A0E0B0E05F
:10714000281739074A075B0718F4868D8460868FF5
:10715000E0915D04F0915E0484A195A1A6A1B7A180
:10716000820F931FA41FB51F80A791A7A2A7B3A743
:1071700080915B0490915C04B9010E9480301F9162
:107180000F910895A0E4B0E0E8ECF8E30C94D44F3C
:107190008091540480FF1AC0E0915D04F0915E0478
:1071A000868D80FF09C080A591A5A2A5B3A584A363
:1071B00095A3A6A3B7A30AC08160868FE0915D0462
:1071C000F0915E0414A215A216A217A2E0915D042C
:1071D000F0915E04868D80FD08C1E0915B04F09122
:1071E0005C04108280915B0490915C0463E978E018
:1071F0000E941448E0915D04F0915E0461A172A1C7
:1072000082E040E050E000E010E020E030E00E944A
:10721000AB0A7B018C016115710581059105C9F1EE
:1072200080915B0490915C046DE77AE00E941448C1
:1072300080915B0490915C04DC010D900020E9F7E3
:107240001197A81BB90B2DB73EB7285030400FB689
:10725000F8943EBF0FBE2DBFEDB7FEB731968A0F33
:107260009B1FADB7BEB712969C938E9311978CEB74
:107270009AE093838283E482F582068317830E94D7
:10728000C749EDB7FEB738960FB6F894FEBF0FBEEC
:10729000EDBF20915D0430915E04F901A1A1B2A17E
:1072A0009C9182E1989FF0011124EF59FE4F859146
:1072B0009491892B09F470C080E0BD0120E030E09A
:1072C00040E050E000E00E946F0AE0915D04F09120
:1072D0005E0461A172A180E0AE014F5F5F4F00E4E8
:1072E00010E020E030E00E94AB0AE0915D04F091F4
:1072F0005E0461A172A180E020E030E040E050E057
:1073000000E00E946F0A89818F3159F48A818B389D
:1073100041F480915B0490915C0461EF79E00E94FC
:107320001448E0905B04F0905C04D7010D900020BD
:10733000E9F78D01015010400E191F09CE01019689
:107340003DDB00D000D000D0EDB7FEB73196E00EA7
:10735000F11EADB7BEB71296FC92EE92119729EAD4
:107360003AE033832283958384830E94C7498091C6
:107370005B0490915C04FC01DF010D900020E9F7B3
:107380001197AE1BBF0BEDB7FEB736960FB6F8944C
:10739000FEBF0FBEEDBF25C0D90193962C912835B5
:1073A00039F480915B0490915C0467E079E00BC054
:1073B00080915B0490915C04233519F466EB78E0CE
:1073C00002C06EED78E00E94144880915B049091B9
:1073D0005C04FC01DF010D900020E9F71197AE1B62
:1073E000BF0BBD010E9480300BC082FF08C080919E
:1073F000540482FD04C080E18093540401C06BDE1C
:10740000C05CDF4FE6E00C94F04F8091540480FFA5
:1074100007C0E0915D04F0915E04868D8160868FE7
:10742000E0915D04F0915E04968D90FD23C0E091A3
:107430005B04F0915C04108280915B0490915C0489
:1074400063E978E00E94144880915B0490915C04A9
:107450006CE379E00E94144880915B0490915C0495
:10746000FC01DF010D900020E9F71197AE1BBF0B67
:10747000BD014DC08091540482FD3BC092FF04C009
:1074800080E18093540435C0CF018196ED5AFF4FBF
:10749000BF0140E350E013DA9C014FEF873F9407B0
:1074A0003CF486EF9FEFAC01421B530B9A010EC0D8
:1074B0000996099720F480E1809354040895E0919F
:1074C0005D04F0915E04868D8460868FE0915D049A
:1074D000F0915E04E20FF31FED5AFF4F8AE08083C4
:1074E000E0915D04F0915E04E20FF31FEC5AFF4F50
:1074F000108280915D0490915E048D5A9F4FFC0133
:1075000001900020E9F73197E81BF90BBF010C94BB
:107510008030A0E0B0E0EFE8FAE30C94D34FEC0148
:10752000E0905D04F0905E0481E290E0E80EF91EC8
:1075300002E380E2D82E1DC0853229F08B3291F40F
:10754000F701D08211C01B811B82CE01019660E041
:1075500070E040E150E00E94DA46F70160831B834F
:10756000229602C0F701808301500894E11CF11CAF
:1075700021968881882319F00023F1F60CC000239E
:1075800051F0F7011082E0915D04F0915E0485E016
:107590009AE390A3878FCDB7DEB7E7E00C94EF4F67
:1075A0008091540480FF03C080E180935404809153
:1075B000540483FD43C0E0915B04F0915C041082AD
:1075C00080915B0490915C04DC010D900020E9F750
:1075D0001197A81BB90B00D000D000D0EDB7FEB7B3
:1075E00031968A0F9B1FADB7BEB712969C938E93B0
:1075F00011978FE49CE09383828380915D04909146
:107600005E048396958384830E94C74980915B04BE
:1076100090915C04FC01DF010D900020E9F71197C7
:10762000AE1BBF0B2DB73EB72A5F3F4F0FB6F89486
:107630003EBF0FBE2DBFBD010C9480300895CF9387
:10764000DF938091540480FF27C0E0915D04F091A6
:107650005E04868D80FD03C08160868F06C082FF38
:1076600004C080E18093540445C1E0915D04F09131
:107670005E0481A192A1B396BF010E94F819E09126
:107680005D04F0915E04882321F4868D8460868FEA
:1076900003C083A18E3249F3E0915D04F0915E0452
:1076A000868D80FD92C0E0915B04F0915C041082B5
:1076B00080915B0490915C0463E978E00E94144837
:1076C00080915B0490915C046EED78E00E94144818
:1076D00080915B0490915C04DC010D900020E9F73F
:1076E0001197A81BB90B00D000D000D0EDB7FEB7A2
:1076F00031968A0F9B1FADB7BEB712969C938E939F
:10770000119781EC9AE09383828380915D0490913C
:107710005E048396958384830E94C749C0915D046B
:10772000D0915E04EDB7FEB736960FB6F894FEBF63
:107730000FBEEDBF8BA1882309F4CDC0FE01B39627
:10774000DF010D900020E9F7AE1BBF0B1297AC0FC5
:10775000BD1F93968C9193978F3211F493961C9240
:1077600080915D0490915E0483966FE270E00E94C8
:107770009648FC01118280915B0490915C04DC01CD
:107780000D900020E9F71197A81BB90B00D000D08D
:1077900000D0EDB7FEB731968A0F9B1FADB7BEB7CD
:1077A00012969C938E93119784E49BE0938382833B
:1077B00080915D0490915E048396958384830E94FA
:1077C000C749CDB7DEB726964BC0C0915B04D091B8
:1077D0005C0482FF0AC0188280915B0490915C0473
:1077E00062E87BE00E94144876C0188220915D0414
:1077F00030915E042D5B3F4FF9018081235430406E
:10780000C0915B04D0915C04A9014D5D5F4F84FF82
:107810002DC0DE010D900020E9F71197AC1BBD0BC8
:107820008DB79EB708970FB6F8949EBF0FBE8DBF59
:10783000EDB7FEB73196CA0FDB1FADB7BEB71296D4
:10784000DC93CE9311978EE19CE0938382835583E2
:107850004483578346830E94C749CDB7DEB7289635
:107860000FB6F894DEBF0FBECDBF35C0DE010D9060
:107870000020E9F71197AC1BBD0BEDB7FEB73C97A5
:107880000FB6F894FEBF0FBEEDBF3196CA0FDB1FD7
:10789000ADB7BEB71296DC93CE9311978BEE9BE0FB
:1078A0009383828355834483578346832A5B3F4F68
:1078B000E90188819981AA81BB8180879187A2870C
:1078C000B3870E94C749EDB7FEB73C960FB6F89450
:1078D000FEBF0FBEEDBF80915B0490915C04FC0184
:1078E000DF010D900020E9F71197AE1BBF0BBD0122
:1078F0000E948030DF91CF910895FC01DB018081EF
:10790000882321F101C0319680818032E1F3882300
:10791000E9F01C920DC09C919295907F9C932081E0
:10792000822F80538A3008F08750892B8C933196B0
:107930009081892F80538A3070F3892F90E08F7D5A
:10794000907081549040069730F302C0E0E0F0E080
:10795000CF010895A2E0B0E0E0EBFCE30C94D14F3E
:10796000DC016B01B42E8FEF8A8301C011968C91DC
:107970008032E1F3873629F0833709F0C5C0EE2461
:1079800004C0EE24E39401C011968C918032E1F79B
:1079900001C0DF01FD0181918032D9F3808190E047
:1079A0008F7D90708434910581F0853491052CF49D
:1079B0008134910509F0A8C00EC08934910539F0D1
:1079C0008F34910509F0A0C004C011E007C010E099
:1079D00005C012E003C0FD01349613E031968081AA
:1079E0008032E1F390E08F7D90708E349105B4F792
:1079F000CF01BE016F5F7F4F80DF009709F484C025
:107A00004981413041F0413058F0423071F043300B
:107A100009F07AC00FC023E230E0E6E0FE2E0EC08F
:107A200020E230E07DEFF72E09C026E230E06CEF77
:107A3000F62E04C029E230E053EAF52E1330E9F4C3
:107A40002DB73EB72A5030400FB6F8943EBF0FBE58
:107A50002DBFEDB7FEB73196ADB7BEB71296DC922B
:107A6000CE921197B282138285E79CE0958384833E
:107A700046831782F094F08620C0B901610F711D12
:107A80008B01EE2041F1DB018C91EDB7FEB73A9707
:107A90000FB6F894FEBF0FBEEDBF3196ADB7BEB7BF
:107AA0001296DC92CE921197B282138225E73CE0C7
:107AB0003583248346831782808711860E949949E3
:107AC000282F30E0EDB7FEB73A960FB6F894FEBF18
:107AD0000FBEEDBF1BC0BE016F5F7F4F0EDF009773
:107AE00099F0BE016E5F7F4F08DFD8012C919A811B
:107AF0008F2D892380958223298192239F21892B91
:107B00008C9320E030E002C02FEF3FEFC9012296B6
:107B1000E9E00C94ED4FFC01DB0180818823A1F0AA
:107B20002181222389F0822F90E0C8971CF02FEF4B
:107B30003FEF5BC080917C002053807F282B2093F7
:107B40007C0058E060E008C050E060E080917C007C
:107B5000807F852B80937C0080917A008064809365
:107B60007A0080917A0086FDFCCF209178003091D8
:107B70007900832F9927482F4F708F7090700A9744
:107B800018F4842F805D02C0842F895C8C93C90116
:107B900044E0969587954A95E1F7482F4F708F708E
:107BA00090700A9718F4842F805D02C0842F895C3E
:107BB00011968C931197822F8F702F7030702A300E
:107BC000310510F4805D01C0895C12968C93129788
:107BD00080E213968C93139714961C926C5F5F5FF0
:107BE000583008F4B3CF262F30E0C901089561154D
:107BF0007105D9F12DB73EB7205130400FB6F8943A
:107C00003EBF0FBE2DBFEDB7FEB73196ADB7BEB7C5
:107C100012969C938E93119785E89CE093838283C0
:107C2000758364836F5F7F4F778366836F5F7F4F5A
:107C3000718760876F5F7F4F738762876F5F7F4F4A
:107C4000758764876F5F7F4F778766870E94E849F3
:107C50002DB73EB7205F3F4F0FB6F8943EBF0FBE23
:107C60002DBF069711F480E008958FEF0895A7E0E7
:107C7000B0E0EDE3FEE30C94D24FFC017B016A011E
:107C800001C0319680818032E1F38E010E5F1F4F7B
:107C90008823F1F0CF01B801AADF87FF03C02FEFDF
:107CA0003FEF51C080E090E0B80146E050E00E9414
:107CB000AD080E949208898382E190E0BE016F5F67
:107CC0007F4F41E050E00E94AD0820E030E03BC033
:107CD000C80160E070E046E050E00E94414E8DB780
:107CE0009EB742970FB6F8949EBF0FBE8DBFEDB7FB
:107CF000FEB73196ADB7BEB71296FC92EE921197D1
:107D0000D382C28289EA9CE0958384838A818683B8
:107D100017828B81808711868C81828713868D8163
:107D2000848715868E81868717868F81808B118A3E
:107D30000E9499499C018DB79EB742960FB6F89460
:107D40009EBF0FBE8DBFC9012796E8E00C94EE4F91
:107D5000A3E0B0E0EEEAFEE30C94D44F8B017A018D
:107D60002DB73EB72A5030400FB6F8943EBF0FBE35
:107D70002DBFEDB7FEB73196ADB7BEB712969C9347
:107D80008E9311978CEC9CE093838283CE010196B5
:107D900095838483CE01029697838683CE010396D2
:107DA000918780870E94E8492DB73EB7265F3F4FF5
:107DB0000FB6F8943EBF0FBE2DBF8A8199818823EC
:107DC00011F4905E01C0985C998389816B810E9457
:107DD00099108DB79EB708970FB6F8949EBF0FBE47
:107DE0008DBFEDB7FEB73196ADB7BEB712961C93F7
:107DF0000E931197F382E28287EC9CE09583848353
:107E00008B81868317820E9499492DB73EB7285FE0
:107E10003F4F0FB6F8943EBF0FBE2DBF2396E6E04E
:107E20000C94F04FA2E0B0E0E8E1FFE30C94D44FF3
:107E30008B017A012DB73EB7285030400FB6F89429
:107E40003EBF0FBE2DBFEDB7FEB73196ADB7BEB783
:107E500012969C938E9311978AED9CE09383828374
:107E6000CE01019695838483CE0102969783868303
:107E70000E94E8492DB73EB7285F3F4F0FB6F894F0
:107E80003EBF0FBE2DBF8A819981882311F4905E79
:107E900001C0985C998389810E94A610ADB7BEB7D6
:107EA00018970FB6F894BEBF0FBEADBFEDB7FEB7C3
:107EB000319612961C930E931197F382E28225ED70
:107EC0003CE035832483992787FD909597838683AB
:107ED0000E9499492DB73EB7285F3F4F0FB6F894DF
:107EE0003EBF0FBE2DBF2296E6E00C94F04FA4E0FB
:107EF000B0E0EDE7FFE30C94D44F8B017A012DB78E
:107F00003EB72A5030400FB6F8943EBF0FBE2DBF8B
:107F1000EDB7FEB73196ADB7BEB712969C938E9370
:107F2000119787EE9CE093838283CE01019695831F
:107F30008483CE01029697838683CE010396918730
:107F400080870E94E8499981892F87502DB73EB7D5
:107F5000265F3F4F0FB6F8943EBF0FBE2DBF893747
:107F600018F02FEF3FEF28C04B815C81892F6A8189
:107F70000E94BC0FADB7BEB718970FB6F894BEBF3E
:107F80000FBEADBFEDB7FEB7319612961C930E93A0
:107F90001197F382E28220EE3CE0358324839783BD
:107FA00086830E9499499C018DB79EB708960FB6AB
:107FB000F8949EBF0FBE8DBFC9012496E6E00C94D5
:107FC000F04FA3E0B0E0E7EEFFE30C94D44F8B0159
:107FD0007A012DB73EB72A5030400FB6F8943EBF15
:107FE0000FBE2DBFEDB7FEB73196ADB7BEB7129637
:107FF0009C938E93119787EF9CE093838283CE01AD
:10800000019695838483CE01029697838683CE0161
:108010000396918780870E94E8499981892F87502C
:108020002DB73EB7265F3F4F0FB6F8943EBF0FBE49
:108030002DBF893718F02FEF3FEF27C0892F6A81B6
:108040004B810E94E80FADB7BEB718970FB6F894F2
:10805000BEBF0FBEADBFEDB7FEB7319612961C93F3
:108060000E931197F382E28220EF3CE03583248364
:10807000978386830E9499499C018DB79EB7089685
:108080000FB6F8949EBF0FBE8DBFC9012396E6E0E0
:108090000C94F04FA2E0B0E0E0E5F0E40C94D44F93
:1080A0008B017A012DB73EB7285030400FB6F894B7
:1080B0003EBF0FBE2DBFEDB7FEB73196ADB7BEB711
:1080C00012969C938E93119787E09DE09383828311
:1080D000CE01019695838483CE0102969783868391
:1080E0000E94E8499981892F87502DB73EB7285FB4
:1080F0003F4F0FB6F8943EBF0FBE2DBF893718F023
:108100002FEF3FEF26C0892F6A810E940A10ADB77A
:10811000BEB718970FB6F894BEBF0FBEADBFEDB790
:10812000FEB7319612961C930E931197F382E2825A
:1081300020E03DE035832483978386830E9499491C
:108140009C018DB79EB708960FB6F8949EBF0FBEE0
:108150008DBFC9012296E6E00C94F04FA2E0B0E09A
:10816000E4EBF0E40C94D44F8B017A012DB73EB7C9
:10817000285030400FB6F8943EBF0FBE2DBFEDB76C
:10818000FEB73196ADB7BEB712969C938E931197FA
:1081900084E19DE093838283CE010196958384835D
:1081A000CE010296978386830E94E8499981892FA0
:1081B00087502DB73EB7285F3F4F0FB6F8943EBFAC
:1081C0000FBE2DBF893718F02FEF3FEF26C0892F44
:1081D0006A810E942310ADB7BEB718970FB6F89406
:1081E000BEBF0FBEADBFEDB7FEB7319612961C9362
:1081F0000E931197F382E2822DE03DE035832483D4
:10820000978386830E9499499C018DB79EB70896F3
:108210000FB6F8949EBF0FBE8DBFC9012296E6E04F
:108220000C94F04FA2E0B0E0E8E1F1E40C94D44FFC
:108230008B017A012DB73EB7285030400FB6F89425
:108240003EBF0FBE2DBFEDB7FEB73196ADB7BEB77F
:1082500012969C938E93119781E29DE09383828383
:10826000CE01019695838483CE01029697838683FF
:108270000E94E8499981892F87502DB73EB7285F22
:108280003F4F0FB6F8943EBF0FBE2DBF893718F091
:108290002FEF3FEF26C0892F6A810E945B10ADB798
:1082A000BEB718970FB6F894BEBF0FBEADBFEDB7FF
:1082B000FEB7319612961C930E931197F382E282C9
:1082C0002AE13DE035832483868317820E94994901
:1082D0009C018DB79EB708960FB6F8949EBF0FBE4F
:1082E0008DBFC9012296E6E00C94F04FA1E0B0E00A
:1082F000ECE7F1E40C94D44F8B017A0100D000D06C
:1083000000D0EDB7FEB73196ADB7BEB712969C93CD
:108310008E9311978EE29DE093838283CE01019626
:10832000958384830E94E8499981892F87502DB7CE
:108330003EB72A5F3F4F0FB6F8943EBF0FBE2DBF2A
:10834000893718F02FEF3FEF24C0892F0E94821049
:10835000ADB7BEB718970FB6F894BEBF0FBEADBF8E
:10836000EDB7FEB7319612961C930E931197F382D8
:10837000E28227E23DE03583248386831782D9D7C2
:108380009C018DB79EB708960FB6F8949EBF0FBE9E
:108390008DBFC9012196E6E00C94F04FEF92FF9259
:1083A0000F931F93CF93DF93EC018B017A018881A8
:1083B000833219F083E28883198289816FE70E94F2
:1083C000940F282F2F5F2983215027FF03C020E01F
:1083D00030E028C08DB79EB70A970FB6F8949EBFBD
:1083E0000FBE8DBFEDB7FEB73196ADB7BEB71296D3
:1083F0001C930E931197F382E28281E39DE09583B3
:108400008483268317822087118693D726EF3FEF38
:10841000281B390B8DB79EB70A960FB6F8949EBFEE
:108420000FBE8DBFC901CDB7DEB7E6E00C94F04FAB
:10843000A6E0B0E0EEE1F2E40C94D64F8B01CE0161
:1084400001960E949D11882319F420E030E02DC090
:108450008DB79EB70C970FB6F8949EBF0FBE8DBF19
:10846000EDB7FEB73196ADB7BEB712961C930E931B
:10847000119788E49DE093838283898184831582A8
:108480008A819B81978386838C819D819187808758
:108490008E81828713867BD79C018DB79EB70C9601
:1084A0000FB6F8949EBF0FBE8DBFC9012696E4E0BB
:1084B0000C94F24FCF93DF93FC0180818823D1F09D
:1084C000EF012196CE0161E67DE042E050E0DFD58C
:1084D000892B11F480E009C0CE016DE57DE043E019
:1084E00050E0D5D5892B31F481E00E94F61520E0CB
:1084F00030E002C02FEF3FEFC901DF91CF91089527
:10850000CF93DF93FC0180818823D9F0EF0121967E
:10851000CE0169E67DE045E050E0B9D5892B11F444
:1085200081E009C0CE0164E67DE044E050E0AFD5D3
:10853000892B39F480E061E00E949A1520E030E058
:1085400002C02FEF3FEFC901DF91CF910895A2E064
:10855000B0E0EDEAF2E40C94D84F2DB73EB72850C6
:1085600030400FB6F8943EBF0FBE2DBFEDB7FEB73B
:108570003196ADB7BEB712969C938E9311978FE646
:108580009DE093838283CE01019695838483CE01FF
:108590000296978386831CD72DB73EB7285F3F4F3F
:1085A0000FB6F8943EBF0FBE2DBF029719F02FEF04
:1085B0003FEF09C00E94A61589816A8141E00E94AF
:1085C000701520E030E0C9012296E2E00C94F44FEF
:1085D000A9E0B0E0EEEEF2E40C94D64FFC0101907D
:1085E0000020E9F73197E81BF90B7A9708F450C09F
:1085F0002DB73EB7265130400FB6F8943EBF0FBEA0
:108600002DBFEDB7FEB73196ADB7BEB711968C93BF
:10861000918385E79DE093838283CE0101969583C4
:1086200084838E010E5F1F4F17830683CE0103964E
:10863000918780870E5F1F4F13870287025010407B
:10864000CE01059695878487CE0106969787868703
:10865000CE010796918B808BCE010896938B828BEF
:10866000CE010996958B848BB3D62DB73EB72A5E83
:108670003F4F0FB6F8943EBF0FBE2DBF099741F490
:108680008981B80141E00E94771520E030E002C006
:108690002FEF3FEFC9012996E4E00C94F24FA4E0DC
:1086A000B0E0E5E5F3E40C94D84F1C821B822DB7B3
:1086B0003EB7285030400FB6F8943EBF0FBE2DBFD6
:1086C000EDB7FEB73196ADB7BEB712969C938E93B9
:1086D000119780E99DE093838283CE010196958373
:1086E0008483CE0103969783868372D62DB73EB7D7
:1086F000285F3F4F0FB6F8943EBF0FBE2DBF892BAA
:1087000099F029813A812430310570F48B818131CF
:1087100020F080E190E09C838B83822F6B810E940C
:10872000E31420E030E002C02FEF3FEFC9012496B0
:10873000E2E00C94F44FFC0101900020E9F731973E
:10874000E81BF90B329718F42FEF3FEF08C0609148
:10875000410470914204019673D520E030E0C901D4
:1087600008950F931F93FC0180818823C1F0CF01EE
:108770001DD4082F843018F02FEF3FEF18C060E0B1
:108780000E94E31410E0609141047091420480E281
:1087900090E02AD51F5F1031B1F7802F03C00E94EF
:1087A000A21580E060E00E94E31420E030E0C901FF
:1087B0001F910F910895FC0101C031968081803294
:1087C000E1F3CF010E945127282F30E03095219509
:1087D0003F4FC9010895ABE2B0E0E1EFF3E40C9440
:1087E000D24F8C017B016A0120913B0430913C0403
:1087F00021153105C1F400D000D000D0EDB7FEB78F
:108800003196ADB7BEB712967C936E931197538392
:10881000428381EA9DE0958384838BD59C01EDB7EB
:10882000FEB736964DC0DC018C91853031F0C90120
:108830000E94BC1885E0F801808380913B049091F0
:108840003C04BE016F5F7F4F0E94F819882319F422
:1088500020E030E03AC089A184FD03C020E230E08E
:1088600002C02FE230E08DB79EB70E970FB6F89496
:108870009EBF0FBE8DBFEDB7FEB73196ADB7BEB789
:108880001296FC92EE921197D382C28286E99DE005
:1088900095838483CE0101969783868331872087D1
:1088A0008CA19DA1AEA1BFA182879387A487B58724
:1088B00040D526EF3FEF281B390BEDB7FEB73E96AC
:1088C0000FB6F894FEBF0FBEEDBFC901AB96E8E04E
:1088D0000C94EE4FA5E0B0E0E0E7F4E40C94D64F42
:1088E000FC0101C0319680818032E1F38E010E5F80
:1088F0001F4F8823F9F0CF01B8010E9496308823DA
:1089000019F02FEF3FEF26C08EE090E0B80144E071
:1089100050E00E94AD080E949208898382E190E0B5
:10892000BE016F5F7F4F41E050E00E94AD0820E044
:1089300030E010C080911D0690911E069B838A83B3
:1089400080911F06909120069D838C83C8010E9410
:10895000CE309C01C9012596E4E00C94F24FA5E0CD
:10896000B0E0E5EBF4E40C94D64FFC0101C0319685
:1089700080818032E1F38E010E5F1F4F8823F9F072
:10898000CF01B8010E949630882319F02FEF3FEFF6
:1089900026C08AE090E0B80144E050E00E94AD08B3
:1089A0000E949208898382E190E0BE016F5F7F4F51
:1089B00041E050E00E94AD0820E030E010C080911E
:1089C0002106909122069B838A83809123069091B1
:1089D00024069D838C83C8010E94CE309C01C9016E
:1089E0002596E4E00C94F24FA5E0B0E0EAEFF4E461
:1089F0000C94D64FFC0101C0319680818032E1F3A6
:108A00008E010E5F1F4F8823F9F0CF01B8010E943D
:108A10009630882319F02FEF3FEF26C086E090E0D4
:108A2000B80144E050E00E94AD080E94920889839A
:108A300082E190E0BE016F5F7F4F41E050E00E9415
:108A4000AD0820E030E010C0809125069091260608
:108A50009B838A8380912706909128069D838C832F
:108A6000C8010E94CE309C01C9012596E4E00C9417
:108A7000F24F0895CF93DF9380912108882309F462
:108A80007AC0109221088091390490913A0401969D
:108A900090933A04809339049FB7F8948091F40539
:108AA000882311F081E004C088E08093F40580E021
:108AB0009FBF882309F05FC00E943F09809139045D
:108AC00090913A046AE070E00E947F4F892BC9F4CC
:108AD000CFE5D4E0D0935E04C0935D0482E00E94B1
:108AE0003F2A8091460490914704892B21F00E94EF
:108AF0008B320E94F70EC957DF4F85E0C43FD8077D
:108B000049F78091390490913A0462E370E00E9441
:108B10007F4F892B11F40E94B80D809139049091F8
:108B20003A0464E670E00E947F4F892B11F40E94A2
:108B30006A0A8091390490913A0464EF71E00E94CE
:108B40007F4F892BB1F410923A04109239040E949D
:108B50000227882361F000D08AE59FE0EDB7FEB7D9
:108B60009283818395D30F900F900E94E0260E94FC
:108B7000A4331092F405DF91CF9108950E94540917
:108B80000E94780E77CF0E94330D0C945A380E94C1
:108B9000490F0E941E090E943E090E941D0A0E9460
:108BA000680A0E948A110C94A615CF93DF93BC012A
:108BB0008230910510F462E070E0A0912408B09139
:108BC0002508ED01E0E0F0E040E050E021C08881C0
:108BD00099818617970769F48A819B81309719F0EC
:108BE0009383828304C09093250880932408FE0118
:108BF00034C06817790738F44115510519F0841706
:108C0000950708F4AC01FE018A819B819C01E90172
:108C10002097E9F641155105A9F1CA01861B970B6A
:108C2000049708F4BA01E0E0F0E02AC08D919C912D
:108C3000119784179507F9F46417750781F4129654
:108C40008D919C911397309719F09383828304C080
:108C50009093250880932408FD0132964FC0CA01E5
:108C6000861B970BFD01E80FF91F61937193029723
:108C70008D939C9343C0FD01828193819C01D90116
:108C80001097A1F68091220890912308892B41F436
:108C900080911301909114019093230880932208EE
:108CA00040911501509116014115510541F44DB700
:108CB0005EB78091110190911201481B590B2091D0
:108CC00022083091230824173507B0F4CA01821B0B
:108CD000930B8617970780F0AB014E5F5F4F8417A9
:108CE000950750F0420F531F5093230840932208DA
:108CF000F9016193719302C0E0E0F0E0CF01DF91F0
:108D0000CF910895CF93DF93009709F450C0EC0101
:108D100022971B821A82A0912408B09125081097EF
:108D200009F140E050E0AC17BD0708F1BB83AA830E
:108D3000FE0121913191E20FF31FAE17BF0779F4C5
:108D40008D919C911197280F391F2E5F3F4F3983CA
:108D5000288312968D919C9113979B838A8341154A
:108D6000510571F4D0932508C093240820C01296B1
:108D70008D919C911397AD01009711F0DC01D3CF39
:108D8000FA01D383C28321913191E20FF31FCE17F1
:108D9000DF0769F488819981280F391F2E5F3F4FC3
:108DA000FA01318320838A819B8193838283DF91BF
:108DB000CF910895A0E0B0E0E0EEF6E40C94C94F46
:108DC000EC012B016A016115710519F0FB0191831A
:108DD0008083C114D10449F0C6010297839728F01B
:108DE00020E030E040E050E0DAC0A9908A2D90E029
:108DF000FDD0892BD1F7FDE2AF1621F4A9903324E1
:108E0000339405C08BE2A81609F4A9903324C11449
:108E1000D10421F0E0E1CE16D10411F5F0E3AF1654
:108E200069F48881883711F0883541F4A980229649
:108E300082E0382A20E1C22ED12C12C0C114D10404
:108E400079F4E0E3AE1659F199E9E92E99E9F92EA2
:108E500099E9092F99E1192F8AE0C82ED12C3AC03F
:108E6000FAE0CF16D10491F080E1C816D10429F0C0
:108E7000E8E0CE16D104F9F415C0BFEFEB2EBFEF3A
:108E8000FB2EBFEF0B2FBFE01B2F24C0A9E9EA2E5A
:108E9000A9E9FA2EA9E90A2FA9E11A2F1BC0F8E0C7
:108EA000CF2ED12CEFEFEE2EEFEFFE2EEFEF0E2FA9
:108EB000EFE11E2F0FC09601442737FD4095542F38
:108EC0006FEF7FEF8FEF9FEF0E94A64FC901DA018E
:108ED0007C018D0120E030E040E050E060E03601B0
:108EE000882477FC8094982C70EDB72EBA0CF9E0AA
:108EF000FB1570F48A2D81548A3118F499ECB92E3F
:108F000006C08A2D81568A3140F589EAB82EBA0CFE
:108F10008B2D90E08C159D0504F56F3FE1F0E21676
:108F2000F30604071507B0F0CA01B901A4019301C3
:108F3000C7D79B01AC018B2D90E0A0E0B0E0280FDB
:108F4000391F4A1F5B1F281739074A075B0710F0B4
:108F500061E001C06FEFA990C7CF4114510451F0F7
:108F6000662311F0219703C031FE04C02297F2015D
:108F7000D183C08330FE07C0509540953095219530
:108F80003F4F4F4F5F4F67FF0AC082E290E09093E0
:108F90002D0880932C082FEF3FEF4FEF5FEFB901C3
:108FA000CA01CDB7DEB7E1E10C94E54FFC0188279B
:108FB0009927E89421912032E9F3293010F02E30DE
:108FC000C8F32B3239F02D3231F4689403C0B9D094
:108FD000820F911D219120532A30C8F31EF49095E1
:108FE00081959F4F0895F8940C94055091118AC66D
:108FF000803219F089508550D0F70895FB01DC01CB
:1090000004C08D910590801921F441505040C8F75B
:10901000881B990B0895FB01DC0102C005900D929D
:1090200041505040D8F70895FB01DC010D9000201D
:10903000E9F7119705900D920020E1F70895FB01E3
:10904000DC0105900D920020E1F70895FC010590E8
:109050000020E9F7809590958E0F9F1F0895FB01E2
:10906000DC014150504088F08D9181341CF08B35EB
:109070000CF4805E659161341CF06B350CF4605E1D
:10908000861B611171F3990B0895881BFCCFFB01BE
:10909000DC014150504030F08D910590801919F459
:1090A0000020B9F7881B990B0895FB01DC0102C071
:1090B00001900D9241505040D8F70895DC0101C055
:1090C0006D9341505040E0F70895FC01819186175F
:1090D00021F08823D9F7992708953197CF01089572
:1090E000FB01DC018D91019080190110D9F3990BDE
:1090F0000895FB01DC014150504030F08D9101900A
:10910000801919F40020B9F7881B990B0895FB0109
:10911000DC014150504048F001900D920020C9F709
:1091200001C01D9241505040E0F70895FC0181E0DC
:1091300090E00190061609F4CF010020D1F70197C5
:1091400008957AE0979F902D879F802D910D11248F
:1091500008950F931F93CF93DF938C01EB0100973A
:1091600031F46115710519F420E030E037C081E079
:1091700090E06EE070E0ABD5FC019C01009771F1CE
:1091800080E88383209771F0D387C28781E8838347
:109190008091260890912708892B21F4F0932708C5
:1091A000E093260801151105C9F011870087838116
:1091B000826083838091280890912908892B71F41B
:1091C000F0932908E093280880912A0890912B08B1
:1091D000892B21F4F0932B08E0932A08C901DF9131
:1091E000CF911F910F9108950F931F93CF93DF930A
:1091F0008C01EB018B8181FF1BC082FF0DC02E8192
:109200003F818C819D812817390764F4E881F981B9
:109210000193F983E88306C0E885F985802F0995D5
:10922000892B31F48E819F8101969F838E8302C0AA
:109230000FEF1FEFC801DF91CF911F910F9108959C
:10924000EF92FF920F931F93CF93DF937C018B01DB
:10925000DB0113968C9181FD03C0CFEFDFEF13C0CC
:10926000C0E0D0E00BC0D8011896ED91FC911997A1
:10927000B8010995892B11F0CFEFDFEFF70181914C
:109280007F01882381F7CE01CDB7DEB7E6E0A8C61F
:10929000A0E0B0E0EDE4F9E48BC6FE013596619103
:1092A0007191A0912808B091290813968C91139779
:1092B000886013968C938091280890912908AF01BB
:1092C0009ED0E0912808F09129082381277F2383ED
:1092D0002096E2E089C6AEE0B0E0E0E7F9E466C6D9
:1092E0000D891E898F89988D97FF02C080E090E8D4
:1092F00001979E838D831A83098386E08C839E0168
:10930000255E3F4FCE010196698D7A8DA90177D0F8
:109310004D815E8157FD0AC02F8138854217530762
:109320000CF49A01020F131FF80110822E96E4E04C
:1093300059C6AEE0B0E0EEE9F9E438C60D891E8901
:109340008F89988D97FF02C080E090E801979E83F7
:109350008D831A8309838EE08C839E01255E3F4FA7
:10936000CE010196698D7A8DA90149D04D815E812A
:1093700057FD0AC02F813885421753070CF49A0114
:10938000020F131FF80110822E96E4E02BC6AEE008
:10939000B0E0ECECF9E40AC60D891E898EE08C83FE
:1093A0001A8309838FEF9FE79E838D839E01275E3B
:1093B0003F4FCE0101966F89788DA90120D02F8172
:1093C0003885020F131FF80110822E96E4E00AC6BA
:1093D000AEE0B0E0EDEEF9E4EBC58DE08C838B8977
:1093E0009C899A8389839E01295E3F4FCE01019615
:1093F0006D897E89A90144D32E96E2E0F5C5ABE0E4
:10940000B0E0E4E0FAE4C4C53C012B015A01FC01E0
:1094100017821682838181FD03C06FEF7FEFB9C190
:109420009AE0892E1E010894211C311CF30123812E
:10943000F20123FD859123FF81912F01882309F4F7
:10944000A5C1853239F423FD859123FF81912F0138
:10945000853221F490E0B301C7DEE8CF982FFF24D6
:10946000EE249924FFE1FF15D0F09B3269F09C3285
:1094700028F4903259F0933291F40EC09D3249F0A5
:10948000903369F441E024C052E0F52A84E0F82AE0
:1094900028C098E0F92A25C0E0E1FE2A22C0F7FCA6
:1094A00029C0892F80538A3070F4F6FE05C0989C3D
:1094B000902C1124980E15C0E89CE02C1124E80E85
:1094C000F0E2FF2A0EC09E3229F4F6FC5FC140E4B0
:1094D000F42A07C09C3619F450E8F52A02C09836E1
:1094E00049F4F20123FD959123FF91912F019923D6
:1094F00009F0B8CF892F8554833018F0805283301B
:1095000038F444E050E0A40EB51E5FE359830FC069
:10951000933631F0933779F0933509F052C01FC07C
:10952000F5018081898342E050E0A40EB51E6101FF
:1095300001E010E011C0F501C080D180F6FC03C04D
:109540006FEF7FEF02C0692D70E042E050E0A40EA3
:10955000B51EC601F0D38C015FE7F52213C0F501FB
:10956000C080D180F6FC03C06FEF7FEF02C0692D91
:1095700070E042E050E0A40EB51EC601D1D38C01CC
:1095800050E8F52AF3FE06C018C080E290E0B3016F
:109590002BDEEA948E2D90E008171907B0F30DC06A
:1095A000F601F7FC8591F7FE81916F0190E0B30120
:1095B0001BDEE110EA94015010400115110581F7FE
:1095C000E2C0943611F0993661F5F7FE08C0F50156
:1095D000208131814281538184E090E00AC0F5010D
:1095E000808191819C01442737FD4095542F82E072
:1095F00090E0A80EB91E9FE6F92257FF09C05095CA
:109600004095309521953F4F4F4F5F4FE0E8FE2A40
:10961000CA01B901A1012AE030E0F4D3D82ED21852
:109620003FC0953729F41F2D1F7E2AE030E01DC072
:109630001F2D197F9F3661F0903720F4983509F07F
:10964000A5C00FC0903739F0983709F09FC004C00B
:1096500028E030E00AC0106114FD146020E130E021
:1096600004C014FD166020E132E017FF08C0F501C8
:10967000608171818281938144E050E008C0F501EE
:1096800080819181BC0180E090E042E050E0A40E36
:10969000B51EA101B7D3D82ED2188FE7F82EF1222C
:1096A000F6FE0BC05EEFF522D91438F4F4FE07C0C5
:1096B000F2FC05C08FEEF82202C01D2D01C0192D4D
:1096C000F4FE0DC0FE01ED0DF11D8081803319F413
:1096D00099EEF92208C01F5FF2FE05C003C08F2D6E
:1096E000867809F01F5F0F2DF3FC13C0F0FE0EC04B
:1096F0001E1510F09D2C0AC09D2C9E0C911A1E2D3B
:1097000005C080E290E0B3016FDD1F5F1E15C8F356
:1097100004C01E1510F4E11A01C0EE2404FF0EC0AF
:1097200080E390E0B30160DD02FF1BC001FD03C0D8
:1097300088E790E00EC088E590E00BC0802F867827
:1097400081F001FF02C08BE201C080E2F7FC8DE2F4
:1097500090E0B30149DD05C080E390E0B30144DD52
:109760009A94D914C8F3DA94F101ED0DF11D8081BA
:1097700090E0B30139DDDD20B1F705C080E290E073
:10978000B30132DDEA94EE20C9F750CEF3016681D1
:109790007781CB012B96E2E117C4FC0120FD08C0C4
:1097A00023FD05C022FF02C073836283518340837F
:1097B0000895EF92FF920F931F9344FF02C033E08E
:1097C00011C046FF02C034E00DC0DB01FC01AA0F4E
:1097D000BB1FEE1FFF1F1094D1F76A0F7B1F8E1F58
:1097E0009F1F31E0660F771F881F991F3150D1F7F7
:1097F0007B018C01E20EF11C011D111DA8019701D6
:10980000B701CA011F910F91FF90EF9008950F9338
:109810001F93CF93DF938C01C80198D2EC0197FD81
:1098200006C0E4DB892BC1F7CE01B801D1D2CE014D
:10983000DF91CF911F910F910895A0E0B0E0E2E297
:10984000FCE4AEC3EC01C62E5A01122F7FD2AC014C
:109850008B3219F08D3249F41068CA9409F466C04D
:10986000CE0174D2AC0197FD61C06DEFD62ED1222E
:109870008D2D8073F1F44033E1F4CA9409F442C0B1
:10988000CE0164D2AC0197FD3DC082E0D82A4837B2
:1098900011F0483551F480E4D82ACA9499F1CE01E8
:1098A00055D2AC0199232CF42DC0D6FC02C080E126
:1098B000D82AEE24FF248701242F2053283080F05B
:1098C000D4FC09C02A3060F0D6FE05C02F7D822F5F
:1098D0008151863020F0CA01BE017AD210C02750D3
:1098E000C801B7014D2D65DF7B018C0182E0D82ACC
:1098F000CA9459F0CE012AD2AC0197FFDDCFD1FC3A
:1099000004C014C0EE24FF248701D7FE08C01095C0
:109910000095F094E094E11CF11C011D111DC5019E
:10992000B801A7012D2D39DF81E001C080E0CDB75E
:10993000DEB7EAE051C3A0E2B0E0E0EAFCE42CC309
:109940006C01A62E8A017901FE01319680E2DF01C9
:109950001D928A95E9F770E030E060E040E050E069
:109960004F01A1E0B0E0F6018381F70183FD25916D
:1099700083FF21917F01222309F47CC02E3519F445
:109980004115510569F1872F90E08417950744F43C
:109990002D3551F12D3221F4332329F431E021C04A
:1099A000332309F4622F322F832F8695869586956F
:1099B000F401E80FF11D832F87703D0102C0660C92
:1099C000771C8A95E2F7208126292083361711F427
:1099D00030E007C0361710F43F5FE6CF3150E4CFD8
:1099E00071E04F5F5F4FBFCF332319F08E818062EC
:1099F0008E83772359F0FE0131969E012F5D3F4FF4
:109A0000808180958193E217F307D1F7BB24B3944B
:109A10004E010894811C911CC60198D1AC0197FDA0
:109A200021C0869586958695F401E80FF11D808109
:109A300090E09A012770307002C0959587952A951D
:109A4000E2F780FD04C0CA01B601C2D10BC0011506
:109A5000110519F0D8014D938D01AA94BB24AA20B9
:109A6000D9F602C0BB2031F40115110529F0F80127
:109A7000108202C0EE24FF24C701A096EEE0A8C227
:109A8000A0E0B0E0E5E4FDE487C25C016B013A01CF
:109A9000FC01178216828824DCC0812F90E0A6DAB0
:109AA000892B19F0C501B3DED4C0153249F4F60193
:109AB000F3FC6591F3FE61916F01653259F415E293
:109AC000C50144D197FDD1C0181709F4C2C0B50132
:109AD0007FD1D0C06A3219F0162F00E006C0F3FC27
:109AE0001591F3FE11916F0101E099240EC00260FF
:109AF000692D70E080E090E040E25BDE962EF6019A
:109B0000F3FC1591F3FE11916F01212F20532A30A0
:109B100070F301FD03C099249A9403C0992009F4BD
:109B2000A9C0183621F01C3699F4F6010BC0F601D5
:109B3000F3FC6591F3FE6191683619F06F01162F01
:109B400007C008600460F3FC1591F3FE11916F01EA
:109B5000112309F48FC083E89FE0612F70E0D5D016
:109B6000892B09F487C0802F00FF03C0EE24FF2457
:109B700007C0F301E080F18022E030E0620E731E46
:109B80001E3649F4F5014681578160E070E0C70157
:109B9000202F03DE5EC0133689F481FD02C09924B4
:109BA0009394C501D3D097FD60C0E114F10419F07E
:109BB000F70181937F019A94A1F749C01B3551F4B5
:109BC000C501692DA7019601B6DE6C01009709F069
:109BD0003EC038C0C5011BDE97FD47C01F3641F1AE
:109BE000103728F4143611F1193621F524C0133733
:109BF00019F01537F9F41AC0C501A8D0EC0197FD8A
:109C00000FC0F4D9892B21F0CE01B501E1D008C0F5
:109C1000E114F10419F0F701C1937F019A9461F7FF
:109C2000E114F104A1F0F701108211C0006203C039
:109C3000006101C00064C501692DA701202FFDDD71
:109C4000882329F4F5018381807379F413C000FF20
:109C50008394F501F380F601F3FC1591F3FE119165
:109C60006F01112309F019CF05C0882019F42FEFD7
:109C70003FEF02C0282D30E0C901CDB7DEB7EEE0DE
:109C8000A7C1DC01CB01FC01F999FECF06C0F2BDF2
:109C9000E1BDF89A319600B40D9241505040B8F7AA
:109CA0000895F999FECF92BD81BDF89A992780B5A4
:109CB0000895262FF999FECF1FBA92BD81BD20BD10
:109CC0000FB6F894FA9AF99A0FBE019608950F9379
:109CD0001F93CF93DF93689F8001699F100D789F3A
:109CE000100D1124C8010E94D545EC01009721F008
:109CF00060E070E0A801E2D9CE01DF91CF911F9121
:109D00000F910895992788270895FC01059006165C
:109D100021F00020D9F7C00108953197CF010895AF
:109D2000FC010590615070400110D8F78095909526
:109D30008E0F9F1F0895FC0161507040019001102B
:109D4000D8F7809590958E0F9F1F0895CF93DF933E
:109D5000EC014B8140FF1AC046FF0AC04F7B4B838A
:109D60008E819F8101969F838E838A81282F2BC0AD
:109D700042FF13C0E881F9818081282F332727FD16
:109D800030952115310529F440624B832FEF3FEFC9
:109D90001BC03196F983E88311C0EA85FB85CE01AB
:109DA00009959C0197FF0AC09B812F5F3F4F11F0DF
:109DB00080E201C080E1892B8B83E8CF8E819F8177
:109DC00001969F838E8330E0C901DF91CF91089582
:109DD0009C01FB01838180FF11C086FD0FC09FEFB6
:109DE0002F3F390759F0228380648F7D83838681DA
:109DF000978101979783868330E002C02FEF3FEF72
:109E0000C9010895FA01AA27283051F1203181F1C2
:109E1000E8946F936E7F6E5F7F4F8F4F9F4FAF4F72
:109E2000B1E03ED0B4E03CD0670F781F891F9A1F85
:109E3000A11D680F791F8A1F911DA11D6A0F711D39
:109E4000811D911DA11D20D009F468943F912AE045
:109E5000269F11243019305D3193DEF6CF0108952D
:109E6000462F4770405D4193B3E00FD0C9F7F6CF5E
:109E7000462F4F70405D4A3318F0495D31FD405226
:109E8000419302D0A9F7EACFB4E0A69597958795BC
:109E900077956795BA95C9F700976105710508959B
:109EA0009B01AC010A2E0694579547953795279547
:109EB000BA95C9F7620F731F841F951FA01D0895DF
:109EC000629FD001739FF001829FE00DF11D649F9E
:109ED000E00DF11D929FF00D839FF00D749FF00D2A
:109EE000659FF00D9927729FB00DE11DF91F639FCB
:109EF000B00DE11DF91FBD01CF0111240895AA1B6A
:109F0000BB1B51E107C0AA1FBB1FA617B70710F064
:109F1000A61BB70B881F991F5A95A9F78095909596
:109F2000BC01CD01089597FB092E07260AD077FDC5
:109F300004D0E5DF06D000201AF4709561957F4FBC
:109F40000895F6F7909581959F4F0895A1E21A2EF6
:109F5000AA1BBB1BFD010DC0AA1FBB1FEE1FFF1FCD
:109F6000A217B307E407F50720F0A21BB30BE40B1D
:109F7000F50B661F771F881F991F1A9469F7609564
:109F80007095809590959B01AC01BD01CF0108951E
:109F90002F923F924F925F926F927F928F929F92F9
:109FA000AF92BF92CF92DF92EF92FF920F931F93E7
:109FB000CF93DF93CDB7DEB7CA1BDB0B0FB6F89498
:109FC000DEBF0FBECDBF09942A88398848885F84D8
:109FD0006E847D848C849B84AA84B984C884DF8049
:109FE000EE80FD800C811B81AA81B981CE0FD11D2D
:109FF0000FB6F894DEBF0FBECDBFED010895EE0F92
:0EA00000FF1F0590F491E02D0994F894FFCF16
:10A00E007364002F004E554C4C00302E3220282900
:10A01E000020002E0800003401FFFFFFFF010305A2
:10A02E0007090E10121416181C1EFFFFFFFFFFFF6C
:04A03E00FFFFFFFF22
:00000001FF
